:020000041100E9
:103000007FB50023284C294D03932800217C284AB2
:1030100001F0DBFA002812D103232800217C03AA47
:1030200001F07AFA00280AD1224B039A9A4206D17B
:10303000214B2248E360224B636104B070BD02263D
:10304000217CFE2228001F4B009601F037FA002851
:1030500001D00020F1E71C4BA2899A42F9D1217CD2
:10306000FF222800194B009601F028FA0028F0D121
:10307000E389174A934203D1164B17486361DCE793
:10308000164A9342E5D1164B164A1B68934206D95D
:10309000C02304222800217C9B0001F078FA124B07
:1030A00012486361C9E7C0460462FF1F3C42FF1F2C
:1030B000813700005959530059598320C0BE00116F
:1030C000FD4100111062FF1F595900001262FF1FDD
:1030D00083050000B1410011A0BE0011821500005F
:1030E0002862FF1F87130000B9420011B0BE001113
:1030F000002370B51A4E1B4C30006361637401F0FD
:103100008BF9402323744B2B0CD9CC233821AC22D0
:1031100030009B01217401F03AFA00280AD0002502
:1031200025740CE0FFF76CFF051E08D1237C0433E7
:10313000DBB2E7E70C4B0D4D63610D4BE381236878
:10314000002B08D1002D06D00C222900200008F009
:1031500093FC2B7B6374300001F09CF970BDC0467A
:103160003C42FF1F0462FF1F5142001190BE00113C
:10317000AAAAFFFFF7B5164B0192C318021D002043
:10318000009388235B05D3181B685C1C1AD09CB283
:10319000402C18D88D781E0CAC466746CD782D0291
:1031A0003D43AE4206D1019800280ED110000C70AC
:1031B000240A4C7003249BB20733A343D218009B0C
:1031C0009A42DED3FEBD4432F9E71000FAE7C0466A
:1031D000FC0F0000802213B503000324019189B283
:1031E000520107319B18A14304305A1A88235B050A
:1031F000C3181B68591C03D190429241104016BD60
:1032000099B2402907D80B000733A343C018904256
:10321000ECD30020F3E74430F9E7134B134A1B6863
:10322000126810B5FA24934201D81A00F824104B02
:10323000E4021B689A4210D813000E4A12689A42A0
:103240000ED3013307D1F823DB029C4203D10A4994
:10325000054808F071FC200010BDFC24E402ECE7F6
:10326000FE24E402F7E7C04600C0071100D00711B2
:1032700000E0071100F00711FFFFFF7FF0B59BB0E2
:10328000150004900391402A00D9A0E006AB5980B4
:103290001A80FFF7C2FF0400042816D9002206A9ED
:1032A000FFF768FF052810D906AB1B88AB420CD18D
:1032B000002D07D0514B2A000499C01808F05CFA81
:1032C000002802D101201BB0F0BD06AB1D802000FC
:1032D0000699FFF77FFF041E7BD1069B0793FFF73C
:1032E0009CFF80235B01C618802307001B039E42BE
:1032F00001D3F826F60288235B05F31801931B68B7
:10330000013302D0019808F04FFC3D49019808F0C4
:1033100013FC3B1D0293331D05938822029B52052B
:103320009B181B6808935A1C3CD044219AB2009108
:10333000402A04D80320D11D814389B2009103990A
:103340001B0C8B4224D0402A22D80122300008A92D
:10335000FFF710FF021E1BD1380008A9FFF70AFF74
:103360000400042831D9009A059B9B188022520141
:10337000B218934240D288235B05C118009A09A86D
:1033800008F07AFB1D4B009A09A9F01808F0A4FA7E
:10339000009A029B9446634402931A4B029AFB18CC
:1033A0009A42BAD388235B05FC1821680198013939
:1033B00008F0C2FB200008F0F7FB039A07AB5A8025
:1033C00030000799FFF706FF0400002C03D100200E
:1033D00079E70428FBD988235B05E018069908F0F3
:1033E000ABFB0323EA1C9A4300D16BE7034B049920
:1033F000E01808F071FA65E70424ECE70400001116
:10340000FFFFFF7FF80F0000F7B505001400402A0A
:1034100021D8002701AE71803780FFF7FEFE042817
:1034200016D93A003100FFF7A5FE042810D93688D6
:10343000BC420BD0BD4209D0221CB44200D9321C80
:10344000064B92B2C118280008F016FB30B2FEBD40
:10345000C04300B2FBE703204042F8E7040000113C
:1034600037B5042204000D0001A81649FFF7CCFF70
:10347000020004280BD1019BA34208D3AB4204D025
:10348000104901A80195FFF7F9FE01203EBD0E4C41
:1034900023682000019308F087FB0199200001397F
:1034A000019108F049FB80235B01E418074B9C4223
:1034B000EED10422034901A80195FFF7DFFE0020A9
:1034C000E4E7C0465555000000C007110000081190
:1034D00030B589B008F0E0FB10226946254808F0B5
:1034E0000BFC254B009A9A420ED1019B029A0F2B9E
:1034F00033D8002101240698013B08D2002900D0CE
:103500000292029B013331D10023029325E0551C26
:10351000F2D102002100EFE710341022200004A9AC
:1035200008F0EAFB029B013301D1069B029388233A
:1035300004995B05C918059B06981A03120B0491A0
:103540000592814203D02B4201D108F095FA019BEC
:10355000013B0193019B002BDED1029B002B03D08A
:10356000049304984168084709B030BDE025014C38
:103570002D03EFE700000111504859368022F8B5BD
:10358000964C974BD200002120001C6008F034FBC1
:103590002300944A88331A60934B1A786A23002ACE
:1035A00000D01133E3620A232365904B37221B7846
:1035B0000820A3638E4B2118E361102323628D4BF7
:1035C0003B256361C823DB00A36123008C331A60B1
:1035D0002823013AE26320646364CA67043A211D28
:1035E000CA672100BC310D602100C0310860210094
:1035F000C4310B6021000635CC310D602100083D3F
:10360000C8310D602100D0310A602200D432106030
:103610002200D832136022000227E0322100176016
:103620004222DC310A6021001B3DE4310D602100A3
:10363000E83108602100EC310B6023000521F433F0
:1036400019602300F0331A602300183290331A6097
:1036500023009433186023001E3A98331A60AF2376
:10366000DB002360644BFA262363644B644DE36004
:10367000644BF031A3642300FF31FC33B600A1603A
:1036800021611E60A5627325E5656D3D6565A565D3
:1036900096255D4AAD00E264666258606766A5667D
:1036A00000270925A767E566584F594D6067200038
:1036B0002567E2673A6015279C30676007001A208B
:1036C00038602000A0300700212038602000A8309A
:1036D00007004C4838602000F83006602600642758
:1036E000A436376026005F3FAC3637602600033FC4
:1036F000B03637602600C637B4363760260000275C
:10370000B836376038269E60424E96205E64424E40
:103710005A66DE61414E9A645E62F53EFF3E9E62ED
:103720001E269A67354A8000DE661F675F67DD6583
:103730001D661862DA67BE23394A5B00E250394BD6
:10374000D838235004302250C4225200A350C6233C
:10375000E4205B00E1500433334AE1503349344BF9
:10376000D1603449800019503349E938FF38195085
:1037700032490430195032493248D161324911631B
:10378000324951631900F4310860CE2030494000BD
:1037900011603049195019002F48F83108602F493D
:1037A000D16582212E4A89005A501A002D490832CB
:1037B000D1671A002C49B432116088212B4A890044
:1037C0005A501A002A49883211602A4ADA6408F0ED
:1037D000C3F8012008F0A0F9F8BDC0460004FF1F9F
:1037E000B464FF1F806FFF1F7444FF1F4A0AFF1F4E
:1037F0003A07000080C3C9019A020000DC050000FE
:103800006A18000050C3000088130000F009FF1F71
:10381000204E00006509FF1F68100000C409000069
:1038200040420F0010270000FC00FF1FB51CFF1FC7
:103830000000FF1F092DFF1F9130FF1F292FFF1FC1
:103840007520FF1F6527FF1F9120FF1F3D22FF1FCF
:103850000120FF1F8929FF1F712AFF1F9119FF1FD8
:103860009528FF1FB925FF1FC525FF1F011FFF1F3B
:10387000B91FFF1F791EFF1F0223F0B50124604D01
:10388000604E2B70604B91B01C70604F0393336897
:1038900000212000BB7006F06DFE200006F064FDE4
:1038A0000023984205D0BA78552A02D0332A00D096
:1038B00099E03360042006F0C5FF08F07DF9FFF7BA
:1038C0005DFE08F069FA1F2201240021504B10AE62
:1038D0001A70504B1C70504B1970504B1968914323
:1038E000163A0A431A60602219689143403A0A4323
:1038F0001A6008F0D9F807F047FF494B9847C120F4
:10390000FF21484B80001A588A431A50C522920062
:1039100098588843BF390143995098584249084004
:103920008021C9010143802099509958C00509029E
:10393000090A0143995080213C48490107F07CFF66
:10394000032322003A49019400933A4808F03CF8D6
:103950002C22394905A808F08FF805AC6178207849
:10396000023406F021FDA642F8D1344C344B2268D3
:1039700003201A40A023DB02134323608023226824
:103980009B041343236022682E4B1A4080239B0321
:10399000134323602C4A2D4B934200D8012008F09A
:1039A0000BF808F039F980232268DB041343236005
:1039B000287807F0A1FF039B1878C0B208F02CF814
:1039C00007F0E2FF2249042007F046FF06F006FF59
:1039D00000F040F800F02EFE00F0D6FE00F016FADF
:1039E000002011B0F0BD00932100194A042007F017
:1039F0008BFF8023DB059C62FFF76AFD5AE7C04618
:103A00004A0AFF1F34F000407444FF1F3462FF1F56
:103A1000480AFF1F490AFF1F680AFF1FBCF0004049
:103A2000E1A2000000E100E0FF00FFFF7844FF1F7B
:103A3000FC56FF1F7854FF1FB8BD001114F0004062
:103A4000FF7FF8FFFFFF9FFF0080FF1F806FFF1FBA
:103A50003B000108002210B51100112008F03CF9CC
:103A600010BD0000F8B500230926364F364C3B62E6
:103A7000E3681120B343E36007F0BEFF112008F0B4
:103A8000B3F8112008F000F84023226810251343F2
:103A9000236080236268DB02134363608023A26893
:103AA00002211343A360A368284A08201340A3609F
:103AB0008023A2689B0113430122A360236CAB43C4
:103AC0002364236C1343236480231B013B62226B1A
:103AD0001F4B1A402263626B1A406263A26B1A404A
:103AE000A263E26B1340E363E3681A4A1340E360A6
:103AF00006F05AFC0121082006F06AFD8023164AD0
:103B00005B00516C11200B43536407F07DFEFD21D7
:103B1000C720124B124A89005A50A36B80002B43D6
:103B2000A363E3680F4A3343E3600F4B1958114016
:103B3000802212020A431A50802292051A600B4B0F
:103B40005D63F8BD00F000403CF00040FFFFDFFF88
:103B5000EFFFEFFFFFFF7FFF003800400000FF1F77
:103B60005118FF1FFF00FFFF00E100E000000540CB
:103B7000E12010B5C00407F0B7FE10BD70B52B4CA6
:103B8000238C002B2AD0FA22D200934201D2FFF7D5
:103B9000EFFF228A238C002A21D1DA00238263825C
:103BA000A382E38223836383A383E383226062602F
:103BB000A260E2601E4D1F4A6420EB8093420AD847
:103BC000FA220020D200934205D91B4A0A219818F4
:103BD00007F072FFC0B200232872238470BD072053
:103BE000E11CCA7F01320240CA7705D10325201D9E
:103BF000C17F01312940C17708325200A35200230E
:103C000021001A00088A01321B180231082AF9D152
:103C1000221DD27F9200A350626823689B18A2687D
:103C20009B18E2689B185B099BB2C3E77461FF1F96
:103C30001C62FF1FB70B000030F8FFFF30B503A870
:103C400004880B20002C0ED14968074D087849786C
:103C5000090201430A20A94205D10121200019804F
:103C6000024B1B7A137030BD192A00001C62FF1F23
:103C7000F7B5150008AA16884A680F4F14785278CD
:103C8000120222430A24BA4214D10122DBB2019269
:103C900000962A0007F0F2FC041E0BD1074B1B68AC
:103CA000002B07D068782A78000210434242504126
:103CB000013098472000FEBD02290000A061FF1FCF
:103CC00030B5012503790400BFB02B4211D00A4959
:103CD000408807F03FF828420BD0084B01A95B8DC4
:103CE0004D800B80064B00221B7A60880B7104F01C
:103CF00023F93FB030BDC0469861FF1FB040FF1FA1
:103D00001C62FF1F10B50549054806F0D9FF0421C4
:103D1000044A054806F096FF10BDC0469861FF1F93
:103D2000FFFF0000E4BD0011B040FF1F10B50248C6
:103D300004F084FF10BDC046C13C00110123037094
:103D40000B4B1A7A4270022282709A78C270DA782B
:103D50000271032242711A7982715A79C2710C225E
:103D600002729A794272DB7983720B207047C046E7
:103D70001C62FF1F022310B50370013B4370053323
:103D8000837010330371443B43712A33837144338E
:103D9000C37100230372064B04001B8843720A3070
:103DA000FFF7CCFF831D0A30C0B2E37010BDC046E0
:103DB0001C62FF1F10B5142007F0CEFE124B142218
:103DC0000021186007F018FF002007F095FE012081
:103DD00007F08AFE022007F057FD032004F0D2F915
:103DE000042006F0E7F9052003F010FC062004F09B
:103DF000DDF8072001F0B2FA082006F003FF0920E1
:103E000001F08CF810BDC046A461FF1F07F02CFE26
:103E1000012007F081FF07F0C7FF0000094B10B534
:103E20000400984205D0012904D12000064906F07B
:103E300047FF10BD0229FCD1013904F0BDFE002866
:103E4000F3D0F6E7FEFF0000CA61FF1F70B50D7AE0
:103E5000100004AA2C00168810221440154220D10C
:103E6000002E20D10A78022A18D14A685178157894
:103E70000E4A09022943914205D00D4A914209D0C8
:103E80001C800A2404E014220A491A8007F0F4FD79
:103E9000200070BD0C2208491A80F7E71C8001241D
:103EA000F6E70824F4E70B24F2E7C046F3FF00002E
:103EB000F4FF00000043FF1FDCBE001110B504003A
:103EC0000749084806F0FCFE074804F0F7FD00200B
:103ED000E40704D50721054A054806F0B3FE10BDE6
:103EE000CA61FF1FFFFF00001D3E001128BE001128
:103EF000F440FF1F00B50C4BBFB01A780B4902A865
:103F000000F0FCFC6B4680B2D880002809D06A46DD
:103F1000074B01A91B889380064B0022188804F0E8
:103F20000BF83FB000BDC046A861FF1FA961FF1F8D
:103F30004E41FF1F5842FF1F00B50C4BBFB01A780F
:103F40000B4902A801F03EFF6B4680B2D8800028E2
:103F500009D06A46074B01A95B8D9380064B00226E
:103F6000188803F0E9FF3FB000BDC046D261FF1FD3
:103F7000D361FF1FF440FF1F5842FF1FF7B50E002B
:103F8000377A1C0008AB11003D001A8820231D4021
:103F90001F423CD13378022B3BD173681F785B788A
:103FA0001B023B431E4FBB4208D01E4FBB4214D0E6
:103FB0001D4DAB4221D00A252800FEBD002A2AD182
:103FC000142C2AD82200F06807F056FD174B1C70FD
:103FD000012CF1D9FFF7B0FFEEE7002A1BD1202C0E
:103FE0001BD82200F06807F047FD114B04211C701C
:103FF000104B187807F0A0FEDEE7E3B20124009230
:1040000001940A00310007F039FB0500D4E70825C8
:10401000D2E70125D0E70B25CEE70D25CCE7C0463A
:10402000F3FF0000F4FF000002290000D261FF1F2F
:10403000A861FF1F5462FF1F332310B504000370F3
:104040000A220749013007F017FD064B0F201B68B5
:104050001A0AE37222731A0C1B0E6273A37310BD4B
:104060001C62FF1F4462FF1F30B501250379040065
:10407000BFB02B4213D00B49408806F06BFE28429C
:104080000DD06A46084B02A81B889380FFF7D4FF27
:104090006B46D8800022608801A903F04DFF3FB035
:1040A00030BDC046CA61FF1F4E41FF1F10B5024818
:1040B00004F0C4FD10BDC0466940001170B5160083
:1040C00004AA148805AA15784A6850781178000265
:1040D0002A4A0843801805284BD807F04DFC0313E3
:1040E0001E29343F0720032C0BD80422121BAA429E
:1040F00000D92A0022491A803000091907F0BCFCB7
:10410000002070BD0720112CFBD81222121BAA42DE
:1041100000D92A001B491A80EEE707200E2CF0D8A0
:104120000F22121BAA4200D92A0017491A80E3E77E
:104130000720032CE5D80422121BAA4200D92A002A
:1041400012491A80D8E70720032CDAD80422121B60
:10415000AA4200D92A000E491A80CDE70720032C75
:10416000CFD80422121BAA4200D92A0009491A807A
:10417000C2E700220A201A80C3E7C046DCD5FFFF51
:1041800073BE0011F061FF1F63BE00115EBE00111F
:1041900059BE001154BE001110B50D21024A03484A
:1041A00006F050FD10BDC04648BE00116441FF1F1F
:1041B00013B5104C0423217C01AA00F0ADF90028AE
:1041C00015D16B469A88236852BA92B2534322891A
:1041D00009491B0C9B184B806B46DA88636852BAFE
:1041E00092B2534362891B0C9B188B8016BD012031
:1041F000FCE7C0460462FF1F1C62FF1F13B5124C90
:1042000006236A46217C00F087F9002819D16B4605
:104210001988236849BA89B24B4321890B4A1B0C80
:104220005B1853806B46D97803335B781B020B43D2
:104230005BBA61689BB24B4361891B0C5B1893802E
:1042400016BD0120FCE7C0460462FF1F1C62FF1F71
:1042500037B5174C07236A46217C00F05DF900282A
:1042600024D16B461B787F2B20D86B46DD78F0235A
:104270002A041B031A406B469B880E495BBA9BB20B
:104280001A4323682D09534322891B0C9B184B802A
:104290006B465A789B7812031B011A4363682A43C2
:1042A000534362891B0C9B188B803EBD0120FCE7A9
:1042B0000462FF1F1C62FF1F7FB50226154C0022FF
:1042C000217C03AB0096050000F0F8F8002802D02E
:1042D000012004B070BD0E23217C0122280000962D
:1042E0006B4400F0EBF80028F2D16B469A89236802
:1042F000D2BA5343228908491B149B184B806B4642
:10430000DA89636852BA92B2534362891B0C9B18D4
:104310008B80DEE70462FF1F1C62FF1F70B5184C24
:10432000237C002B0FD0382B0ED1164D280000F027
:1043300073F8CC23AC222800217C9B0100F027F9E4
:10434000280000F0A7F870BDE3890F4A934209D115
:104350000C4D280000F060F800222800217C00F0BD
:1043600005F9EDE7094A9342EDD1064D280000F02A
:1043700053F890222800217C920100F026F9DFE713
:104380000462FF1F3C42FF1F8305000083200000E2
:1043900070B5144C237C002B1FD06369002B1CD0FC
:1043A000114D280000F038F8636928009847040090
:1043B000280000F06FF8002C10D10C4B0422995EFD
:1043C000002905DA9C801A8801321A80200070BD0D
:1043D000074A9142F7DD9A80F5E70124FEF788FE4F
:1043E000F4E7C0460462FF1F3C42FF1F1C62FF1F30
:1043F0000F27000010B58024064AA4001168436B03
:10440000234205D113685B1A032BF8D9012010BD94
:104410000020FCE76008FF1F70B5C17905000C00A3
:10442000631E9C411A4BE402E41849000460C9B2BF
:10443000007906F003F9E979687949000131C9B2D8
:1044400006F0FCF8E8790930C0B207F01DFB002344
:10445000E36661332360AA795B3B002A0ED02268B1
:104460009A43023B134323600A23E3610733236229
:1044700000232363A3630133E36370BD22689A437F
:10448000022313432360462363610633A361EFE7EE
:104490000050004070B5002504000368DD66C07957
:1044A0000930C0B207F0A8FA2900207906F062F8B6
:1044B0002900607906F05EF870BD0000F8B51E00B6
:1044C00006AB1D78002304681700E366616007F0FF
:1044D000E3FB01238022E3662B0027615200013BAE
:1044E00008D207F011FC08200A4A1168002D03D1F8
:1044F0002800F8BD2261F2E7236F034203D023694D
:10450000013D3370013613685B1A032BEED9012588
:10451000EEE7C0466008FF1F70B51C000023056869
:104520001600EB66696007F0B7FB01238022EB669B
:1045300023005200013B08D207F0E6FB08200A4A9C
:104540001168002C03D1200070BD2A61F2E72B6FA7
:10455000034203D02B69013C3370013613685B1AA8
:10456000032BEED90124EEE76008FF1F002370B58E
:1045700004681500E366616007F08EFB0123E366C3
:10458000256107F0C1FB2000FFF734FF70BD70B557
:104590001D00002304681600E366616007F07CFBE1
:1045A0000123E36626610F33626B1A42FCD02B0AAB
:1045B00023611023626B1A42FCD0EDB2256107F033
:1045C000A3FB2000FFF716FF70BD002370B5046841
:1045D0001500E366616007F05FFB0123E3662B0AC9
:1045E00023611023626B1A42FCD0EDB2256107F003
:1045F0008BFB2000FFF7FEFE70BD70B51E00002390
:1046000005681400EB66696007F046FB0123A619F4
:10461000EB660F33B44205D107F076FB2800FFF7B5
:10462000E9FE70BD21782961696B1942FCD0013423
:10463000F0E7000010B5084CE368002B08D1802299
:10464000064B52021B689B186360054B1B68236076
:1046500007F08AFBA06010BD4462FF1FC8F0004055
:10466000CCF0004070B5184A936A916A9942FBD128
:1046700016498A689A421FD39A1A8B60144B0126F6
:10468000186893B2D202D20E4343424300204C68D2
:104690001B0A1B1912029B180E4C0A684B60551C12
:1046A000A3420CD8002801D04B600A600A4A13606C
:1046B00008680A4B186070BD581E821ADDE7084A68
:1046C00030009B182A00EAE700F000404462FF1F18
:1046D000140AFF1F40420F00C8F00040CCF0004019
:1046E000C0BDF0FF70B51F4C23793F2B01D93F238C
:1046F00023711D4B22791A701878C0B207F044FA62
:1047000018231A491A4A0B801A4913800B805380C8
:10471000A379194980200B800C21938001334B43EE
:10472000164D191C0001834200D9011C2980D1803B
:104730006379002B01D101336371237A012B01D8F6
:10474000022323726279237A0D4853430A21584386
:1047500007F0B2F90B4D2860E379052B01D810233F
:10476000E37170BD3862FF1F480AFF1F5642FF1FEA
:104770002044FF1F5442FF1F5242FF1F5042FF1FA1
:10478000710200002862FF1FF8B520210020FEF70B
:1047900067FE114C011E114D09D10C22104BC1CBEB
:1047A000C1C4280007F028FAFFF79CFFF8BD0C22CF
:1047B00020000C49FEF728FE0C2802D0084B43CB02
:1047C00043C40C2228000849FEF71EFE0C28EBD03B
:1047D0000C220021E5E7C0463862FF1F0462FF1F7C
:1047E000D0BE0011FC0C0000F50C0000F0B51D4C13
:1047F0008022A5440400882069465201400507F044
:10480000E3F9902212016A441300200032C832C337
:1048100016C816C38023144C144FA6689B03334359
:10482000A3603B6007F0E0F88823A0685B05C01830
:1048300007F0BAF90025882329008022A0685B05CB
:10484000C01840196944520007F046F8802301352A
:10485000FF355B019D42EED1A6603E60044B9D4456
:10486000F0BDC046FCEFFFFF9043FF1F9808FF1FFD
:1048700004100000F0B5040087B0002825D0684679
:1048800007F0DAF81B4C022806D106226946200000
:1048900006F072FF002816D06946002301250F2676
:1048A0002F00E25C013310091030874038002F00E0
:1048B000324097403A0002434A610439062BEFD157
:1048C0006846FFF793FF07B0F0BD182269460A4813
:1048D00007F07AF96A46A300D358013305D01822AD
:1048E000FF21684607F088F9EAE70134062CF1D188
:1048F000E9E7C0466509FF1F00090011F0B5002572
:1049000004000E0085B0AA4200D186E04B1C087856
:1049100001934B788978377909021943F3783F0678
:104920001B040B431F43039720706570252800D19B
:1049300096E033D8112813D806F006FF69003A0133
:104940003A013A013A01AA00B800B1003A013A012D
:104950003A013A013A013A013A013A0114013401AB
:10496000232800D1EDE0DB2800D043E1042A00D861
:10497000B1E01025052A05D0551F2A003800711D09
:1049800007F07AF805223100200007F075F82A00B8
:104990003900601D07F070F805353EE0562859D003
:1049A00010D8332800D1A7E0552839D02628DAD1ED
:1049B000A64B2900132218001D0007F01DF9FEF771
:1049C00097FB5CE0712800D177E0722800D189E084
:1049D000602800D195E0DC28C5D1022A00D87AE011
:1049E0007378BFB26370B378A370032A05D0033A1B
:1049F000390092B2F01CFEF741FC10223900E01C95
:104A0000FEF702FDC51C002807DA607070E00C227A
:104A100020008F4907F030F80C25280005B0F0BDC4
:104A2000013A8C4D0C2A13D8002A0AD0280001998B
:104A300007F022F8FFF756FE0C2228008649FEF701
:104A40001DFC29000C22601C07F016F80D25E4E778
:104A50000C22EBE77F4D814B2A0043CB43C2E9E7B1
:104A6000013A7A4D0C2A11D8002A08D00199280061
:104A700007F002F80C2228007949FEF7FFFB290015
:104A80001322601C06F0F8FF1425C6E70C22EDE7A0
:104A900006227449601C06F0EFFF0625BDE71222CE
:104AA0007149601C06F0E8FF1325B6E708226F493C
:104AB000601C06F0E1FF0925AFE7012A0ED07178EE
:104AC000F02908D86A4D288801F0D8FD694B2A885A
:104AD0005200D35A00E0FF23637009E0644A654B3B
:104AE0001288F5E7644B012A04D072785A7062701C
:104AF000022592E75B78EFE72000FFF79DFA0500BB
:104B00008BE7013A5D4D072A07D8002A06D100231A
:104B100001202B6001F0A2F80CE007229621584BEF
:104B200089001B6857485B1801992B6006F0A4FFA9
:104B300001F060F8691D0722601C06F09DFF082542
:104B40006BE7042A04D94E4D2F6007F00DF9A860D9
:104B5000FFF788FD0422039003A9601C06F08CFF78
:104B600005255AE7484D062A15D90622280001993D
:104B700006F002FE00280ED006220199280006F059
:104B80007BFF062241492800FEF778FB01233A4AC1
:104B900051780B43537029000622601C06F06CFF0D
:104BA00007253AE7012A96D07078FFF763FE9FE762
:104BB000012800D0D7E6931E354F132B06D8737803
:104BC000002B0BD100F018F900F04EF9314B3900F1
:104BD0001D78601C6A1E06F04FFF1EE7551E2A0056
:104BE0000199380006F048FF38002B49AAB2FEF7B9
:104BF00045FBE9E7DA281DD1042A00D86BE7082A2B
:104C000015D9B37972791B021343F27912041A434E
:104C1000337A1B0613433B603B68052231002000BA
:104C2000039306F029FF0422601D03A941E7FE2338
:104C30006370F1E7DE2800D04DE7511E012A01D153
:104C40000025EAE6019800F0BBFFF9E70462FF1FC8
:104C5000DCBE00113862FF1FFC0C0000D0BE00114A
:104C6000F50C00001062FF1FF061FF1F9443FF1F4F
:104C70005842FF1FB864FF1F3462FF1F9464FF1F78
:104C80004462FF1F9964FF1F6509FF1FADAC000060
:104C90003564FF1F3364FF1FAEDE000070477047AE
:104CA000020010B5094B0A32094C92B2DA815A82DD
:104CB00098811882207802F047FB0422054B0121DD
:104CC00020781A7007F038F810BDC0461E43FF1F49
:104CD0007E64FF1F7D64FF1F013870B5042809D86A
:104CE00006F04AFE030928081200234B0221187817
:104CF00007F022F870BD204B0821187806F0E4FE7A
:104D000000221E4B1A72F5E7802200241B4B1A4D1D
:104D100052001A8108211A682878DC7206F02CFFEC
:104D20002100287806F000FF012000F063FE00F06B
:104D300061FFDFE7104B0821187806F0C5FE104828
:104D4000FFF718F80F4B104A9B79002093800F4A09
:104D500013808022094B5200D8721A8100F04AFE5B
:104D600000F048FF0A4B5B78002BC3D0094A136060
:104D700006F03AFDBEE7C0465462FF1F2862FF1FDF
:104D80006142FF1F3862FF1F2044FF1F5242FF1F76
:104D90003462FF1F34F0004010B500290BD1012808
:104DA00009D1054B1B78002B05D02622034B044864
:104DB0005A72FFF775FF10BD5664FF1F2862FF1F70
:104DC000C40900000300F0B50A4D8E18B14202D1AB
:104DD00052008018F0BD0C782F6824093C5D0F2725
:104DE0001C700C7801313C402F683C5D5C700233D4
:104DF000ECE7C0464C42FF1F0D22124B10B51A7053
:104E00000C23114C11492370093A033B104863707D
:104E100006F032FE2D2301220E490F48A371FFF741
:104E2000D1FF01220D49FFF7CDFF01220C49FFF709
:104E3000C9FF030000200B4902001870FEF71EFA9C
:104E400010BDC0465264FF1F3364FF1F73BE0011C4
:104E50003564FF1F6709FF1F3A64FF1F6609FF1FC4
:104E60006509FF1FAEDE000070B5134C1422200050
:104E70001249FEF7C9FA431E114D132B19D8AB780E
:104E8000002B16D0431C2B7009236B7000230019D4
:104E9000037028780B4B01302900C0B2187006F05F
:104EA00043FD297822000139C9B2002005F0E8FD50
:104EB00070BDFFF7A1FFECE73564FF1FAEDE000019
:104EC0003364FF1F5264FF1F10B5114B1A7818701E
:104ED000002A0ED000280BD10E4B1A78062A07D8CC
:104EE0005423D340DB0703D50B4B187802F02CFA80
:104EF00010BD0028FCD0074B1B78012B02D0033BD0
:104F0000022BF5D8044B0121187806F015FFEFE7C6
:104F10005664FF1F7D64FF1F7E64FF1F70B54A4EFD
:104F20004A4A4B493070012005F036FC00F0E8FE9B
:104F3000FEF7DEF806F018FD032246494648FFF763
:104F400041FF2D24030004221C7044490130FFF767
:104F500039FF30230470424D424C437083702E3B26
:104F6000062220004049EB87FEF74EFA062813D0B0
:104F7000200006F061FD022809D00321200006F080
:104F800063FC8D23E3706E3B23711933637106223A
:104F900020003549FEF772F9344B1B68FC335C6422
:104FA000FFF762FF0020FFF78FFF314C314A0121EC
:104FB000314B1278207802F089F9304A304B127860
:104FC0000021207802F082F901222E4B1A702E4B1C
:104FD0009B78552B31D12D4B3B325A722C4B2D4A9D
:104FE000AB81EA812B826A822021307806F05CFE58
:104FF0000120404205F090FD0120404205F02CFECA
:10500000FFF7CAF8FEF77EFE00F0B2FC0120404236
:10501000FEF754FF012006F00FFEF02001F012FB16
:105020000121307806F088FE307802F0E9FA1A485B
:1050300006F092FBFEF716FD70BD6422174B5B79FC
:1050400053431A000A32CBE75462FF1F994D0011F7
:105050009D4C00119443FF1FF061FF1F1062FF1F62
:105060001E43FF1F6509FF1FADAC0000B464FF1FA6
:105070007E64FF1F8042FF1F6142FF1F5264FF1FBB
:105080003364FF1F2464FF1F3462FF1F2862FF1F69
:10509000C4090000CE0900005662FF1F3862FF1FDE
:1050A000F8B50A0020230D001A40194263D05E4B68
:1050B0001B78002B5CD0FFF7D5FA5C4B5C4C5D4E47
:1050C00099686268737A8A1ADB039A4202D3616034
:1050D000FEF7C8FC327A217A531EDBB2994205D121
:1050E000FFF71CF9002000F0B9FD15E09142F9D35B
:1050F00000272772FFF74CF9A37ABB4202D0A772B0
:10510000FEF73CFD012000F0A9FD4B4F3800FEF7F3
:1051100031FE390006F0D8FB637A002B25D0013B25
:10512000DBB26372002B20D1444B9B78552B01D10D
:1051300006F05AFBE37A002B12D00023A27AE37226
:105140009A4202D0A372FEF719FD3D4A3A4F1388E6
:10515000380001331380FEF70DFE390006F0B4FB72
:10516000642370795843FFF79BFD237A0133237240
:1051700020206840F8BD0BB2002B0ADA314B1878BA
:1051800006F02AFD002801D006F0DEFC8020000297
:10519000EFE70224214206D0254B01201A72FFF7C7
:1051A00093FE2000E5E70B071ED5FFF75BFA1F4BC8
:1051B0001F49204C98684A68637A821ADB039A4236
:1051C00002D34860FEF74EFCFFF7E2F8FFF7A6F8BF
:1051D000012000F043FD00F0E5FB2368DB0701D56B
:1051E000FEF764FF0820C4E7CB0609D5FEF7C6FC2E
:1051F0000D4B1B78002B01D1FEF798FD1020B8E76E
:105200000124214207D0104800F06CF806F094FB0E
:1052100000F00AFDC5E70424080020402142A9D07F
:10522000FEF768FEBDE7C0465664FF1F4462FF1FDD
:105230002862FF1F3862FF1F6142FF1F3462FF1F99
:105240001C62FF1F5462FF1F4442FF1FF0B51B4B3F
:105250001B4F1B883A8804001A4E1B4D85B09A429A
:105260000DD832889A420AD3184B1A882B889A4252
:1052700005D1174A174B12881B889A421BD005206C
:1052800001F036FA3B8802AA1380338801905380DC
:105290002B88114D93800F4B02A91B88D3800F4B95
:1052A0002A78188802F052FF0D4B08212878019ABD
:1052B0001C7006F031FB05B0F0BDC0462264FF1F34
:1052C0005642FF1F5442FF1F5242FF1F2064FF1F20
:1052D0001E64FF1F5042FF1F7E64FF1F5842FF1FC6
:1052E0001C64FF1F13B50C4B1C78002C11D1002837
:1052F00001D00A4B18600A4A0A4B11780A4A107802
:105300000A4A01920A4A0092002205F0B1FA2000EE
:1053100016BD1124FBE7C0467D64FF1F1864FF1F04
:105320007C64FF1F6C64FF1F7E64FF1F5864FF1FB7
:105330005C64FF1F10B5064B12201B78052B06D1AD
:10534000044B13221988044B187801F0ADFB10BDF3
:105350007D64FF1F5842FF1F7E64FF1F10B50024AD
:105360000122114B52421870104B1C70104B1A80C6
:1053700002F046F904220F4B21001A700E480C323D
:1053800006F0B2FC102221000C4806F0ADFC07220A
:105390000B4B1C600B4B1C700B4B1C700B4B1A7097
:1053A0000B4B1C7010BDC0467E64FF1F7D64FF1F49
:1053B0005842FF1F7C64FF1F6C64FF1F5C64FF1F6B
:1053C0005864FF1F3264FF1F3164FF1F5A42FF1FE2
:1053D0003064FF1FF8B5174C0600257806A8142482
:1053E0000078052D23D1B41F134FA5B21824BD4258
:1053F0001DD88D1FADB2BD4219D8FA256D00AA4245
:1054000015D21D000D4F0A3DADB2BD420FD80C4C58
:1054100026800C4C21800C4900240A800B4A138002
:10542000FFF714FF0A4B0421187806F04DFB20000B
:10543000F8BDC0467D64FF1F790C0000750C0000AC
:105440005642FF1F5442FF1F5242FF1F5042FF1F90
:105450007E64FF1FF0B50BB20D0089B0002B00DB9E
:1054600070E1A44E307806F0B7FB041E50D00378EC
:10547000A22B00D122E1D02B1AD0912B45D1437819
:105480000E2B42D19C4B82889A423ED19B4A836824
:105490001278052A39D1032018567F2835D0984B29
:1054A0001B68002B31D05B68002B2ED098472CE076
:1054B0008078072829D806F05FFA0428183F3F743F
:1054C000A8D86378002B0CD101218C4B19708D4B1F
:1054D0001A78002A5BD08C4B307801F0F7FE002858
:1054E00055D00722854B1A7051E061780029F8D118
:1054F000E378002B11D0854A854B1278307801F083
:10550000E5FE60706378002BEBD1200006F01CFBF9
:1055100080200002684009B0F0BD784B1B78022B58
:10552000F3D00121307806F08FFA0028EAD101216A
:10553000307806F001FCE5E76378002BD1D16F4F9E
:10554000032807D13B78052B02D101333B701EE0C5
:105550000223FBE76F4B1A886F4B0293002A0BD094
:105560001B78002B03D00121307806F0D5F93B7869
:10557000062B04D1013BE9E7029B1A70F7E7042BE5
:1055800041D10121029B3078197006F0D5FB5C4BAC
:105590001B68002BB9D01B68002BB6D0574A107877
:1055A00084E76378554F002B27D10622211D5B48E5
:1055B00006F062FA62895A4B5A491A80A2895A4BFC
:1055C0001A80E3890B800521397058490A80584AAE
:1055D0001380228A574B1A80574B1B78012B09D115
:1055E0001F2001F085F8FA2292004243042130780E
:1055F00006F092F90022484B75E7312B00D070E796
:105600000022454B1A700323A0E7062200214348DD
:1056100006F06AFB0023454A04211380444A30788F
:105620001380444A138006F04FFA0821307806F0C0
:105630004BFAA379083B5A425341304A0333137063
:10564000304B1B78002B06D0334B30781A78002A69
:1056500006D001F079FE0122314B52421A8096E7C2
:105660000121197006F068FBF5E70821307806F093
:105670002BFA6378002B00D047E72C4B2D4F029379
:10568000E388029A04211380294B307803932389FD
:10569000039A138063893B8006F0D6F9002800D076
:1056A00033E7264B1B68002B00D12EE703990298A5
:1056B0003A88098800881B68984726E74379132BA6
:1056C00000D022E70389012B0AD11D4B1B78022B46
:1056D00006D10821307806F0F7F9FFF72BFE14E722
:1056E000052001F005F808210200307806F014F9D1
:1056F0000BE7C0467E64FF1F051400007D64FF1F9A
:105700001864FF1F8042FF1F6142FF1F5264FF1F8A
:105710003364FF1F5464FF1F5664FF1F2564FF1F7F
:105720005842FF1F2C64FF1F2E64FF1F2264FF1FBF
:105730002064FF1F1E64FF1F2464FF1F1464FF1FEB
:105740001C64FF1F8020C001014200D0E2E6CB07AD
:1057500031D5324B1B78002B1DD0314E05AC337840
:10576000052B1AD1023B23702E4B21001B7823728C
:105770002D4B1B7863722D4B187801F04BFD0028E0
:1057800009D007202A4B30701B68002B03D01B6800
:10579000002B00D098470120BCE60E20254B0622A6
:1057A0001B7825492370254B1B78637002ABC0180A
:1057B00006F062F9D8E7022308001840194209D020
:1057C000174B1B78052B03D11D4B188806F06CF87E
:1057D00002209FE60424214203D0FFF737FD20007A
:1057E00098E6082308001840194200D193E6154BAB
:1057F0001C78012C03D0022C0DD008208AE6124B15
:10580000124A134913481B8812880988008800949B
:10581000FFF7E0FDF1E7FFF78DFDEEE75664FF1FB0
:105820007D64FF1F5A42FF1F3064FF1F7E64FF1F0D
:105830001864FF1F3264FF1F5B42FF1F3164FF1FAC
:105840005842FF1F1C64FF1F5042FF1F5242FF1FA0
:105850005442FF1F5642FF1F10B502A804880B20B8
:10586000002C10D1496808784978090201430C4896
:10587000814209D1022119800A4B59881170DB78C5
:1058800000205BB2537010BD074C0A20A142FAD130
:1058900002211980034B998811705B79F0E7C046AB
:1058A0006E2A00001C62FF1F6F2A0000F7B515006A
:1058B00008AA16884A680F4F1478527812022243B9
:1058C0000A24BA4214D10122DBB2019200962A00C6
:1058D00005F0D4FE041E0BD1074B1B68002B07D02C
:1058E00068782A78000210434242504101309847BC
:1058F0002000FEBD022900009064FF1F30B5012585
:1059000003790400BFB02B4225D01449408805F02C
:1059100021FA28420CD0124B01A95B8D00220B808A
:1059200002234B800F4B5B888B80608802F004FB66
:105930000D49608805F00EFAC0070CD50B4B01A984
:105940001B8800220B8002234B80064B9B888B8098
:10595000608802F0F1FA3FB030BDC0468864FF1F96
:105960008442FF1F1C62FF1F8064FF1FDE42FF1F77
:1059700010B5074C0749200005F0A2F920000649A0
:1059800005F09EF90721054A054805F05BF910BDB1
:10599000FFFF00008864FF1F8064FF1FFCBE001132
:1059A0008442FF1F10B5024803F048F910BDC046FD
:1059B000FD5800110221430888400B400A3108407D
:1059C00003430E20024A117A81430B43137270473E
:1059D0009464FF1F064A537A410705D580210B4383
:1059E00080015372D07270477F210B40F8E7C046A8
:1059F0009464FF1F054A9379002803D080210B434C
:105A0000937170477F210B40FAE7C0469464FF1FF3
:105A10000E22134B197A1140197200281ED0114A18
:105A2000127A502A10D910220A431A722022197AA7
:105A30000A431A724022197A0A431A728022197A8A
:105A400052420A431A7205E03C2AEFD8282AF1D8BC
:105A5000142AF3D80122197A0A431A727047C046F1
:105A60009464FF1F1C62FF1FF8B57F23324D0400B2
:105A7000AE799E43314B984205DD76236B71363B00
:105A80003343AB71F8BD2E4B984203DA58236B7148
:105A90001433F5E783B21A0000215F32294892B22D
:105AA000294F697182422DD9E9718C4203DA5B4238
:105AB0001CB220236B71053420B20A2105F0FCFFD3
:105AC00004B2FA239B009C4233DB80236A795B4259
:105AD00013436B716421200005F0EEFF0A2100B230
:105AE00005F0A2FF09B26A797B5C13436B710A214E
:105AF000200005F0E1FF0A2100B205F095FF09B290
:105B00007B5C0AE08022EA71002CDADA5B421CB28C
:105B100020236B715F23092CE9DC1E430A2120003E
:105B2000AE7105F081FF09B2EA797B5C1343EB713A
:105B3000A8E7632CCEDCEDE79464FF1F1B4E00004A
:105B40001DFCFFFF2A08000026BF00117F23F7B5C8
:105B5000194FCD017E7A04009E437E72EDB2632818
:105B600006DD093B33437B7240231D43BD72F7BD05
:105B70000300093304DA582333437B726C23F4E7C0
:105B80000E4B019300280BDA0423444224B27B72AB
:105B90000A21200005F048FF019B09B25B5CE4E7A5
:105BA0000928F5DD0A2105F087FF019B00B21B5C87
:105BB0001E437E72ECE7C0469464FF1F26BF0011AF
:105BC000F8B50A4F05003B790E00002B0CD0084CAD
:105BD0002000FEF721FC33002A0020003979FEF76F
:105BE0000CFD2000FEF756FCF8BDC0469464FF1F74
:105BF000F842FF1F70B5094D094C0722290020000B
:105C000005F0BAFD002808D029000722200005F081
:105C100033FF08210348FFF7D3FF70BD9964FF1FCE
:105C2000A164FF1FA064FF1F7F2210B50A4B997962
:105C30009143033A5A71103A0A439A7178220E211D
:105C4000DA711A7A8A431A726B225A720C3A9A7271
:105C5000FFF7D0FF10BDC0469464FF1F224A234BBC
:105C600012681B6810B59A4234D3002832D0204CF9
:105C70000223E05E1F4B1B685B062CD509233221F3
:105C8000584305F019FF4130FF3000B2FFF7ECFE3A
:105C90000520FFF78FFE0422A35E174A632093427C
:105CA00005DC32331800642105F006FF00B2012143
:105CB000FFF74CFF0120FFF7ABFE0020FFF78AFE45
:105CC0000E4B1878053843425841C0B2FFF792FE98
:105CD000FFF790FF10BD0A21053005F0EDFE00B280
:105CE000FFF7C2FE0320D4E74462FF1F9464FF1F46
:105CF0001C62FF1F3862FF1FDD2600007D64FF1F4E
:105D000070B50024094D2800AC71FEF785FB102307
:105D10003E212800064AFEF770FCA04200D13E3426
:105D2000044B28001C71FEF7B5FB70BDF842FF1F45
:105D300016BF00119464FF1F0200F0B501270A4846
:105D40000A4E51188B1A002B00DCF0BD0824157880
:105D50004308684038404000805B013C58406D0873
:105D6000002CF5D10132EDE7FFFF000036BF001136
:105D7000F0B500250F269D4200DBF0BD4C5D070904
:105D800044403440A400A05801357840F3E70000B7
:105D9000F0B589B06A460D000B000F2711001035D1
:105DA0001C780133260024093E40167054700232DC
:105DB000AB42F5D12023024AFFF7DAFF09B0F0BD6C
:105DC0003CBF0011F0B54E780B7889B036020C005C
:105DD000170001901E43012A61D9954B9E4200D8BD
:105DE00077E001339E421CD1062A17D1CA788B78FE
:105DF00012021A430B791B0413434A7912061A4301
:105E00008C4B5A6100221A705A808B4A5A608B4A16
:105E10009A608B4ADA60002009B0F0BD88225205F2
:105E2000EEE7884B9E423CD182498B78002B00D014
:105E3000F6E00C2A31D10F22A3789343E2781202C4
:105E400013432279120413436279120613434B6001
:105E5000E279A07912020243207A00041043627AA8
:105E600012060243CA60E27AA07A1202024376481E
:105E70004A81834208D804236E49142201980B708A
:105E800005F0FAFD1420C7E71201D21889235B053B
:105E90009A42F0D801238B70BDE7022AFAD005237D
:105EA000EAE76A4A01239642E6D1FFF743FA052F53
:105EB0000CD9E378A2781B021343227912041A4307
:105EC00063791B061343624A0393136005F08CFC4D
:105ED000A1E7584D2B78002B9DD1AB78002B00D13A
:105EE000A0E02B8901339BB20093B34200D091E034
:105EF000132AD4D9CF7C8B7C3F02122120001F4370
:105F0000FFF71AFF874200D08EE0002E3DD1E378E4
:105F1000A2781B0213432279E96812041A436379B9
:105F20001B06134303930A228B4212D1FF23A37053
:105F3000E370237163716B89002B09D1E37B227CB1
:105F40001B0212041343A27B13431B0901336B8111
:105F500000226B89002B8ED0002A67D16868370138
:105F60003818000B6B6900030390984205D96861EB
:105F700005F01AFEEB780133EB7068681022A11C63
:105F8000381805F0A9FC2E8145E76F89009A7B1E21
:105F90009BB293423AD1E278A37812021A43237952
:105FA00005A81B04134362796C6812061A43EB6858
:105FB00000920392211D0C22049305F05DFD012047
:105FC000260004A940421036FFF7E2FE013F012FF0
:105FD00017D1009A0B232861824200D04CE704229B
:105FE0001C49200005F078FC042203A9686805F02C
:105FF000EBFDE968039AFF23914200D13CE7F73BB0
:106000003AE73100FFF7C4FE1036DFE70923B74255
:10601000A4D831E7009BB34200D9FCE607232BE765
:10602000022329E7032327E7062325E70A2323E79B
:10603000FFFE00000043FF1F00000111FFFF0000F2
:106040005048593601FF0000FFFF001102FF000019
:1060500034F000400C43FF1F10B5034C0B0001222D
:10606000210000F06BFA10BD196200110B8870B5A9
:1060700006000D000224162B11D92B00032209491A
:1060800000F05CFA041E0AD1074B2A881B88191CF1
:10609000934200D9111C300089B200F0EFFA2000C1
:1060A00070BDC04645620011BA64FF1F10B54A7842
:1060B0000400013A0B000220012A07D80A78002ABE
:1060C00004D005222000024900F038FA10BDC04675
:1060D000736200110A7810B50B0004000220002A38
:1060E00004D007222000024900F028FA10BDC04663
:1060F0001F6300110A7810B50B0004000220002A6B
:1061000004D009222000024900F018FA10BDC04650
:106110008563001110B5034C0B000B22210000F029
:106120000DFA10BDB563001110B5034C0B000D2224
:10613000210000F003FA10BD2764001110B5034CD4
:106140000B000F22210000F0F9F910BD816400114D
:106150000A7810B50B0004000220002A04D0112296
:106160002000024900F0EAF910BDC0469164001118
:10617000002310B51322190000F0E0F910BD000053
:1061800010B5034C0B001722210000F0D7F910BD09
:10619000E3640011002310B51922190000F0CEF9B4
:1061A00010BD000010B5034C0B001B22210000F0B5
:1061B000C5F910BD1D650011F7B584890D000600F5
:1061C0000121002C22D000238268D3561778002B9F
:1061D0001EDA0C2C1AD90C3CA4B213194088009377
:1061E000230002F086FE431E984101307B06DB0F40
:1061F0006B703F23013C1F40A4B22870AF70AC808D
:10620000002C07D0B3680133AB6000210800FEBD4D
:106210000020EBE7AC60F8E70B7803704B88437025
:106220004B881B0A83700B79C370042070470420CD
:10623000022B06D10020537811781B02009A0B43E1
:10624000138070470B8803700B881B0A4370022071
:1062500070470420009983420AD1537810781B02BA
:1062600003430B80D37890781B02034300204B80BC
:106270007047F8B50D004B7801240021461C0370CF
:106280002B788B4201D82000F8BD6B78B01C4F1CD6
:10629000012B10D1890069184B88022233704B887A
:1062A000B9001B0A7370691805F0B6FA0436043495
:1062B000A4B2F9B2E4E7122359436B185A880431A7
:1062C00032705B8810221B0A7370691805F0A4FAFB
:1062D00012361234ECE770B5049D14001E00052B35
:1062E00001D8042070BD637812781B0213432B8001
:1062F000E378A2781B02134302226B802A71211DCE
:10630000681D063E05F088FAB2B22A81E92AE8D86B
:106310002800A11D0A3005F07FFA0020E2E70023E3
:1063200010B50A789A4201D8900010BD9A008A18D8
:106330005488013304705488DBB2240A4470948872
:1063400084709288120AC2700430EAE710B5110016
:10635000029C062B04D004201022142B01D010BD67
:10636000022222714B7808781B0203432380CB78EA
:1063700088781B02034363800431601D05F04CFAEA
:106380000020ECE710B50C788B7804315C43E4B264
:1063900003702200013005F03FFA601C10BD04209C
:1063A000022B06D10020537811781B02009A0B4370
:1063B0001380704710B50C000A88023105F02CFAE2
:1063C000208810BD70B504000D0004981100012B49
:1063D00001D8042070BD1678527812023243028030
:1063E0000200F13255701470E125002C00D10C35FB
:1063F000023B9AB24280AA42EBD80231043005F047
:106400000BFA0020E6E70420009983420AD1537872
:1064100010781B0203430B80D37890781B02034350
:1064200000204B80704710B50C000A88023105F03F
:10643000F3F9208810BD000070B501211E00042072
:10644000049C0E400B4218D1CB40DDB28D4214D9D2
:106450000A49DBB2098899420FD32300EE331D703D
:106460003300580011184978165C09023143013392
:106470002152D9B28D42F4D8002070BD1843FF1FBD
:1064800010B50C000A88023105F0C6F9208810BD4D
:1064900010B50C788B7804315C43E4B203702200B1
:1064A000013005F0B9F9601C10BD10B5110002985B
:1064B000032B01D8042010BD14785278043B12023B
:1064C00022430280CA788C781202224342809AB218
:1064D0008280EB2AEED80431063005F09DF90020C9
:1064E000E9E710B50C000B8803700B881B0A43709A
:1064F0004B8883704B881B0AC3708A88043006312E
:1065000005F08AF9A088043080B210BD0420012B68
:1065100003D100201378009A1370704710B50C0057
:106520000B8803700B881B0A43704A8802300431C1
:1065300005F072F96088023080B210BDF0B589B004
:1065400003931E4B029242000700D05A019102F0C1
:1065500020F81325061E2DD0029B01240370019BF9
:10656000002B04D0001903999847001984B26B4698
:106570001B7A5BB2002B0FDA1021380002F01CFBF3
:106580001925002813D130003219E1B202F066FC5F
:10659000051E0CD10C34A4B2042304AA380005A9AA
:1065A00093800696948101F0AFFD051E02D0300065
:1065B00005F012FA280009B0F0BDC046B864FF1F0C
:1065C00070B505000C0000280CD00020814209D0D5
:1065D00010222000044905F01FF901202B782373B5
:1065E0006B78637370BDC0467CBF0011F0B50600C8
:1065F0000D0017001C0085B002291BD000201029B7
:1066000007D1022B07D0102B03D115E00020102C4E
:1066100008D005B0F0BD69463800FFF7D1FF2A0069
:1066200069460BE069463000FFF7CAFF2200694661
:10663000380004E0022BE9D12A003900300005F0CF
:1066400013F9E6E7031CF02800D9F02303200849DA
:106650009AB2013A0B80D317034006499B189B104E
:106660000B80D30F04499B185B100B807047C0460A
:106670001C43FF1F1A43FF1F1843FF1F034B1B88B8
:106680008B4202D3024B4000C15270471C43FF1F94
:10669000B864FF1F014B4000185A7047B864FF1FD1
:1066A0001722014B1A807047B864FF1F70B50500B0
:1066B0000E2005F0D1F9041E13D0D023037000235F
:1066C0000622837007494570033005F0A5F8064B94
:1066D0002100DA8A62811B7E2373044B187805F04F
:1066E00073F870BDD464FF1FC464FF1F6C43FF1FA9
:1066F000262803D8024B4000C05A70470148FCE7E7
:106700001E43FF1FFFFF000070B506000C00094D7F
:106710001C220021280005F0E7FA074B1E70074BEA
:106720001C7005F0B1FA0123002801D000231220CB
:106730002B7070BDC464FF1F6C43FF1FE564FF1F17
:1067400070B505000D4C0800E260A1601022002128
:10675000656005F0B1F8012803D11021A06802F0AE
:1067600058FD10220021280005F0A6F8012803D1C9
:106770001021606802F04DFD70BDC046C464FF1F6B
:1067800070B5041E05D1002903D006220D4805F07E
:1067900043F80D4B1D78012D11D1002C05D102229B
:1067A0001A7005F089FA280070BD00221A70074B94
:1067B0001B78FF2BF7D02000FFF778FFF3E70025C9
:1067C000F1E7C046D464FF1FC464FF1F6C43FF1F82
:1067D000030010B5002801D1002010BD00780B4A3D
:1067E000002803D15988D1821B7913761378022BA4
:1067F000F2D10023984200D103331370044B1B786D
:10680000FF2B01D0FFF752FF0120E6E7C464FF1F12
:106810006C43FF1F002911D000280CD04B790128B0
:1068200003D140225242134303E03F221340032886
:1068300002D001204B7170474022F4E70800FAE7CC
:1068400070B5094D0100287800280BD0074C0622AE
:10685000200004F0E1FF21002878FFF7DBFF200093
:1068600005F01AF870BDC046E464FF1FBE64FF1F48
:1068700000290AD0012808D13F224B799343C02B2D
:1068800003D0403B5A425341981C704770B5174D96
:1068900006002B78FF2B15D00A2005F0DDF8041E2A
:1068A00010D0D0230370C83B8370114B11491B7863
:1068B0004670C3700622043004F0AEFF2100287831
:1068C00004F082FF0C4B1B78012B0DD10B4B1B6886
:1068D000002B03D09B68002B00D09847084B042165
:1068E0001878084A05F048F970BDC0466C43FF1F90
:1068F000E464FF1FBE64FF1FE064FF1F0C65FF1F01
:106900001065FF1F60EA0000014B98687047C046A1
:10691000C464FF1F014BDB6818687047C464FF1F25
:10692000074B10B5DA68136801331360054B18780C
:10693000FF2803D08021C90105F0FEF910BDC04633
:10694000C464FF1F6C43FF1FF7B50E0002F0C8F8C8
:10695000051E1CD00E4B06621F78002F00D1077851
:10696000AB791020019305F077F8041E0FD0D023E7
:106970000380C73B8370019BE91DC370062204306E
:1069800004F04AFF21003800E66004F01DFFF7BD67
:106990006A43FF1F014B18787047C046E464FF1F2D
:1069A000054B002805D1054B1A78054B002A00D16C
:1069B000014B18007047C046D464FF1FE464FF1FFA
:1069C000BE64FF1F014B58687047C046C464FF1F78
:1069D000024B1868431E9841C0B27047E864FF1F1D
:1069E000421E03000120152A03D9FF3B5A4253419E
:1069F000D8B27047F0B51C0000230E0085B003909C
:106A000002920B70029A934201D3002019E0E55CD8
:106A10005A1CD2B2002DF8D0029851198142F4DCF0
:106A20000233DFB2A35C18000193FFF7D9FF0028FF
:106A300007D0013D019A0399EBB233708A4202D12B
:106A4000E01905B0F0BDDB19DBB2DBE710B50C00D7
:106A500002F09EF803001220002B03D0210058887A
:106A600004F0AAFE10BD000070B50E4D84006359FD
:106A7000002B15D0186A002801D005F0FDF82B591D
:106A8000586A002801D005F0F7F82B59986A0028B9
:106A900001D005F0F1F8285905F0EEF800232B514C
:106AA00070BDC046F464FF1F1C4B70B504000E009F
:106AB000150099420AD11A4B1B68002B01D11220F4
:106AC00070BD1B68002BFAD09847F9E7154B994227
:106AD00015D1134B1B68002B0AD01B68002B07D065
:106AE0009847002804D1104B1C70104B1D70E7E72D
:106AF00029002000FFF7AAFF0028E1D1F3E70800F2
:106B000001F0EEFF0028DAD003780320A342D7D1AA
:106B10002900300004F050FED2E7C046FEFF00001E
:106B2000F064FF1FFFFF0000ED64FF1FEC64FF1F18
:106B3000F7B50400808801F0D3FF0025A84203D0F8
:106B40000578A08802F008F81C4E3378002B1FD07F
:106B5000AB421DD11A4B28001978FFF777FF0028A8
:106B600018D000233370A3790820A778A688019352
:106B700004F072FF011E0DD0D0230370CA3B837056
:106B8000019B477086808371280004F01DFE01E0A0
:106B9000002DE8D1A0880B4B8200D358002B01D0E8
:106BA000FFF762FF1721A088FFF768FDA08801F0BA
:106BB00027FDA08801F0FEFDF7BDC046ED64FF1F74
:106BC000EC64FF1FF464FF1FF0B587B01D000CAB31
:106BD0001B88070001930DAB1B88142002930EAB9A
:106BE0001B88160003930FAB1B880091049310AB16
:106BF0001B88059304F030FF041E1AD0D0230370C5
:106C0000CB3B47708370C670062229000430002DEC
:106C100011D004F001FE019B21006381029B0098CA
:106C2000A381039BE381049B2382059BA37404F04F
:106C3000CBFD07B0F0BD05F057F8ECE7F7B50093D2
:106C400008AB1B8807000C200D001600019304F010
:106C500003FF041E13D0280001F042FF00280FD0CC
:106C60000078D0232370C93BA370009B21002381AF
:106C7000019B6770A580E680638104F0A5FDF7BDE8
:106C8000014B1878EDE7C0466C43FF1F13B50400B5
:106C900064890389C2888188C0780094FFF7CEFF99
:106CA00013BD000010B5044C2068002803D004F088
:106CB000E3FF0023236010BDF864FF1FA122F0B59D
:106CC000818892004A43384B384F1B6804009B1858
:106CD0009D2292009B18827989B01A603B68002B34
:106CE0005FD01D78324B1B68002B04D05B68002BF3
:106CF00001D000209847260008363100E079FFF7E0
:106D0000B7FD237DE0710200E0780493638A2900D7
:106D10000393238A0293E3890193A38800933300AA
:106D2000FFF752FFE378002B0BD1E289A379A1880A
:106D300002920196E27928000092012201F0DAFE27
:106D4000E0703B68002B20D0FFF7ACFF194D28788E
:106D500000281AD0184B1978FFF778FE002814D0B5
:106D60002B78E67808200793A78804F075FE011EAB
:106D700009D0D0230370CA3B467083708780867128
:106D8000079804F021FD00232B701721A088FFF73E
:106D900075FCA08801F034FCA08801F00BFD09B05F
:106DA000F0BD064B9DE7C0463409FF1FF864FF1F86
:106DB0000C65FF1FED64FF1FEC64FF1F6C43FF1F9A
:106DC000F8B5070008000E0001F08AFE041E18D076
:106DD0002620FFF78DFC051E00D12578062004F043
:106DE0003BFE041E0DD00021062204F07DFFD023BF
:106DF0002370C23B21006770A370A680E8B204F044
:106E0000E3FCF8BDF0B585B001930AAB1B78070031
:106E100002930BAB1B7808000D000092039301F066
:106E20005FFE061E22D0102004F016FE041E1DD0A8
:106E30001022002104F058FF2620FFF759FC0028FB
:106E400000D13078D0232370C13BA370009B210078
:106E50002372019B67706372029BA580A372039BE0
:106E6000C0B2E3720C9BE36004F0AEFC05B0F0BD71
:106E7000F7B50D00019001F033FE071E20D00E2063
:106E800004F0EAFD041E1BD02620FFF731FC061E8D
:106E900000D13E78D0232380C53B0622A370F91D84
:106EA000E01C04F0B9FC019B2A0063810123DD4052
:106EB0001A401D40210022736573F0B204F084FC77
:106EC000F7BD0000F0B585B0029010000D0017006E
:106ED0000A9E039301F004FE041E31D0029B002B96
:106EE0002ED1039B02795B0724D51223134304227E
:106EF000002E08D10B99002905D10C99002902D147
:106F00000D9900291AD01A430D9B2271002B00D035
:106F1000C9E0002E00D1CFE0002D00D0CCE0606AA7
:106F2000002801D004F0A8FE1C21300004F06CFE03
:106F3000606205E002239A430E33D7E7934323713F
:106F4000654BBA00D458002C00D1AAE0002E10D016
:106F5000236A002B03D11C2004F0FEFD20625E4B4F
:106F6000BA00D358186A002803D01C22310004F05C
:106F700053FC0C9B002B12D0574CBB001D596B6A65
:106F8000002B03D1162004F0E7FD6862BB00E35834
:106F9000586A002803D016220C9904F03DFC0D9B82
:106FA000002B11D04C4DBC006659B36A002B03D1A5
:106FB000142004F0D1FDB0622B59986A002803D048
:106FC00014220D9904F028FC380001F089FD051EFB
:106FD00067D0414BBA00D358002B62D01A6A3420D4
:106FE000002A00D11C389A6A002A01D0143080B2DD
:106FF0000B9A002A01D01C3080B25B6A002B01D0B2
:10700000163080B204F028FD041E4AD01822002158
:1070100004F06AFE2620FFF76BFB0190002801D1E7
:107020002B780193D0232370029B200063700A23E6
:10703000294EA370039BBD00A371AB59A780196AA9
:107040001830002905D01C22A06004F0E5FB2000C8
:1070500034307359996A002907D00300142214337D
:10706000E060029304F0D8FB02980B9B002B08D041
:1070700003001C221C330B992061029304F0CCFB0B
:1070800002987359596A002903D01622606104F0EE
:10709000C3FB6B462100187904F096FB3800FFF71C
:1070A000E3FC05B0F0BD10220D9B0D991B69A018E3
:1070B000236204F0B1FB2CE70B9B002B00D13FE7D0
:1070C000012D00D03CE7606A002801D004F0D4FD17
:1070D0001C210B982AE7C046F464FF1F10B5044C2E
:1070E0002068002803D004F0C7FD0023236010BDF2
:1070F000E864FF1F0B4B07B51A68002A01D1002076
:107100000EBD6946531C012012780731FFF772FC4F
:107110000028F4D002780123100018401A42EED063
:10712000EEE7C0460465FF1FF0B51F4F01203B6826
:1071300087B0002B25D09B78059300F0B3FB002887
:1071400021D00A20FFF7D4FA04000B20FFF7D0FA71
:10715000164B05001E78731E9E413B68F6B2191D42
:10716000D878FFF757FB3B682900DA7A043303929B
:107170009A7901930292009033002000059A04F05E
:10718000E3FD07B0F0BDFFF7B5FF002805D00620EE
:10719000FFF7AEFA04000720D8E70820FFF7A8FAA7
:1071A00004000920D2E7C046E864FF1FE464FF1F23
:1071B00070B50A4E040033780D00FF2B0DD004206B
:1071C00004F04AFC011E08D0D0230370CE3B45706A
:1071D0008370C470307804F0F7FA70BD7C43FF1FF1
:1071E00070B5040006200D0004F036FC011E0AD024
:1071F000D0230370CD3B8370054B44701B688580A2
:10720000187804F0E1FA002C01D0FFF767FF70BD99
:10721000E864FF1FF8B5264F06003B680D001124F7
:10722000002B05D10522234B1B78134202D11224D7
:107230002000F8BD204A10241268002AF8D01278E5
:10724000002AF5D0DB0719D52B789A1E012A1AD807
:107250000C2004F081FC132438600028E8D00023BF
:107260000A22437029000670023004F0D5FAFFF7B5
:107270005BFF041E0AD0FFF731FFD9E700F012FBD5
:107280000028E1D1E4E7002BE2D0D0E70B4B1B78DC
:10729000032BCDD11D20FFF72BFA094B18800028B6
:1072A000C6D0084B04211878074A04F065FCBFE7F4
:1072B000E864FF1FE564FF1F0465FF1FE464FF1F10
:1072C000E264FF1F1065FF1F60EA0000F7B501933D
:1072D000194B14001A78052306000F0012201A42D9
:1072E00021D0012920D1154B1D68002D1BD0022073
:1072F0001F2C18D8002C02D0019B002B13D0104B50
:107300001F221E706E1C0021300004F0EDFC01995C
:107310002200300004F080FA310020002C70002F91
:1073200006D004F001FDFEBD064B12201D68DCE70F
:1073300004F0FAFAF7E7C046E564FF1F0465FF1F93
:107340007C43FF1F0065FF1FF8B50F4E1224336802
:10735000002B17D01B780F3C834213D100250B4F15
:107360000221387804F0B0FB094B042138781D80E5
:1073700004F0AAFB074B28001D8033685C7004F002
:107380002BFA04002000F8BDE864FF1F1065FF1F02
:10739000FC64FF1FE264FF1F70B5012823D11B4C62
:1073A0002388002B03D01A4A1578002D07D0194BDB
:1073B0001B68002B02D01878FFF7C6FF70BD3B2B6F
:1073C00002D93C3B2380F9E7134E0221307804F0C8
:1073D0007BFBFA222388920002215A43307804F082
:1073E0009BFA2580EAE70B4B1B68002BE6D00B4B82
:1073F0001B785B07E2D5084B0221187804F064FB88
:107400000022024B1A80FFF769FED7E7FC64FF1FDA
:10741000E064FF1FE864FF1F1065FF1FE564FF1FA6
:10742000F8B51E4D2868002803D004F025FC002381
:107430002B601B4E3068002803D004F01DFC002395
:107440003360184F05243B7818002040234221D098
:10745000154800F02BFA3B78234213D0202004F08B
:107460007BFB2860002813D02022002104F03CFC84
:10747000202004F071FB041E306005D02022002182
:1074800004F032FC002004E0286804F0F5FB2C60D6
:107490001320F8BD00F00AFAF4E7C0460465FF1FA8
:1074A0000065FF1FE564FF1F7043FF1F10B50A4C06
:1074B00023681A1E0ED0002808D10130587004F03D
:1074C0008BF9002805D02368002B02D00021FFF79C
:1074D00087FE0122100010BDE864FF1FF7B5274E9C
:1074E000050033680191181E21D05C78244F012CCF
:1074F00030D1FFF7FFFD002825D02000FFF7F8F876
:107500000400412814D91F4B022118781E4A04F0A8
:1075100033FB1E4B3C3C1C80022233685A703B7884
:10752000002B14D128000199FFF75AFE0120FEBD5F
:10753000FA2292004243002AEED0124B0221187820
:1075400004F0EAF9E8E7FFF7D3F80200F3E70023D5
:107550003B70EBE73B78002BE8D1032004F07CFA8A
:10756000011E08D0D0230370CC3B45708370336874
:10757000187804F029F9FFF7B1FDD7E7E864FF1F99
:10758000E064FF1F1065FF1F60EA0000FC64FF1F3E
:1075900010B51749838802008B4220D011D81549B5
:1075A0008B4217D0144900205B1899B2012907D8E3
:1075B000926811785A425341D8B2FFF7F9FD012081
:1075C00010BD0E4A00209B1807229BB29A424041F0
:1075D000C0B2F5E783681878FFF768FFF0E78368C3
:1075E00099785A78090218781143FFF777FFE7E78F
:1075F0000A20000006200000F8DFFFFFAFDFFFFFDA
:10760000014B18707047C0467D43FF1F10B5064CF4
:10761000207001F041FA207804F026FB0521207843
:1076200000F062FD10BDC0461065FF1F0BB273B5C0
:107630000D00002B00DBC4E0884B187804F0CCFA76
:10764000041E0ED00378912B0FD0A22B00D1A1E005
:10765000834B1878FF2852D0210004F0B5F8002899
:107660004DD180200002684076BD43780F2B76D044
:1076700013D8052B70D00E2BEAD18088794B984215
:107680002BD8794B98421BD8784B9842E0D1A3680D
:107690001878591CFFF774F838E03E2BD8D183785E
:1076A000032B74D06CD8012B6ED0022BD0D1704B31
:1076B0001B68002B23D05B68002B20D098471EE06E
:1076C0006C4BC0180C28C3D804F056FB1DC2C21561
:1076D0000BC20B0B0B3223C23C00674BC0180728B0
:1076E000B6D8664B1B68002B09D01B68002B06D050
:1076F000200098470AE0A3681878FFF7C7F8200031
:1077000004F022FAADE7A068FFF762F800289FD0E6
:10771000F5E7A3681B78002BF1D0554B1B68002BB5
:10772000EDD01B68002BEAD0210055489847EDE7C3
:107730004F4B1B68002BE2D01B68002BDFD02100D1
:107740005048F3E7504B1B68002BD8D05B68002BE8
:10775000D5D021004348E9E7FFF7EAF9CFE7808871
:107760004A4B984203D04A4B984200D070E7464BB0
:107770001B68002BC3D05B68002BC0D02100D5E76D
:10778000153B012BBBD963E7FFF798FAB7E7FFF783
:107790007DFAB4E73F4B1B78042B07D100236A46E0
:1077A00013800179408800F0C5FCA8E7364B1B68C0
:1077B000002BA4D05B68002BA1D00100364898476D
:1077C0009DE7012421420AD0294B1B68002B04D0DD
:1077D0005B68002B01D000209847012043E78B070E
:1077E0000AD5264B1B68002B04D05B68002B01D008
:1077F00020009847022036E70421280008400D4267
:1078000000D131E7254E3388002B21D0013B9BB2BC
:107810003380002B1AD1FFF7DBF800280AD0204B69
:107820001C70164B1B68002B04D05B68002B01D02A
:1078300020009847FFF7C6F8694601F001FD684649
:10784000FEF7FEFF1D20FEF753FF308004200AE7FD
:10785000024B187804F038F9F8E7C0461065FF1FAE
:107860007D43FF1F0E2000000120000009100000D2
:107870000865FF1FFEDFFFFFAFDFFFFF0C65FF1F87
:107880000C2000000B200000F064FF1F0D20000002
:1078900013200000E564FF1FFFFF0000E264FF1FEC
:1078A000E064FF1F10B501F09BF910BD014B18609B
:1078B0007047C0460C65FF1F0B880020162B01D8AF
:1078C00017230420014A13807047C046BA64FF1F83
:1078D00000207047074A03001188814207D0918831
:1078E0000020994202D1013080001018704700201A
:1078F000FAE7C0461865FF1FF0B58F7806000D0047
:10790000C5B01E2F15D1FFF7E5FF051E03D10024DA
:10791000200045B0F0BD00223B003100C07800924D
:1079200000F0B2FB0400A81C00F0D2FBFF23EB70B8
:10793000EEE7264B062403931B78FF2BE8D0182F85
:10794000E6D87B08224A013BDB0002929A58944613
:10795000002ADDD0029AD3185B68002BD8D00878B3
:10796000002802D14B78012B02D10624122FCFD14F
:1079700007AFAB88697800976446AA68A047041EE1
:10798000C6D1AB78029A5B08013BDB00D318390003
:1079900030005B689847041E0BD1AB78042BB6D03F
:1079A000039A310010782200009700F06DFB04006C
:1079B000AEE76A78002AABD1AA7805A93B8808719E
:1079C00030000A704B80FEF747FBA0E78043FF1FA3
:1079D0008CBF00111D4B37B5050098420BD0002914
:1079E0000AD1FFF777FF002805D11948FFF772FF8A
:1079F000002800D0058037BD01291AD1FFF76AFFA2
:107A0000041EF8D001235B420380A378FF2BF2D041
:107A1000FE2B07D00023E0781422009329001E33A8
:107A200000F032FBA01C00F053FB01235B4263809B
:107A3000E1E70229DFD1013901F0BEF80028DAD1EF
:107A40002800FFF747FF041EDFD1D4E7FEFF000048
:107A5000FFFF0000022210B5074B52421A80074870
:107A600001325A809A80DA8000F07EFA044801F0F0
:107A700025F8002010BDC0461865FF1FF9780011D9
:107A8000D57900110388F7B50400002B02D1022537
:107A90002800FEBD42680221137825485268FEF78F
:107AA000A5FD00282ED0234F01253A88002AEFD0CB
:107AB000802321885B0201259B1A9942E8DC0C2077
:107AC00004F04AF8061E31D03B8822889C460023E9
:107AD0001800019561469DB2491989B2AA421BD886
:107AE000002801D062443A8000233000082208C0F8
:107AF000210003F091FE104A1368002B13D10025DA
:107B00001660C5E76268022113780C485268FEF7D8
:107B10006DFD0028C7D1BAE760681D014019418199
:107B200001330198D6E71A001B68E6E71325AFE793
:107B3000FABF00117E43FF1F1465FF1FF8BF00113D
:107B4000014B18707047C0468043FF1F14230A0082
:107B500010B51A40194204D00122102101F048F852
:107B600010BD4B06F9D4012088434000F8E710B55A
:107B700014008B0604D50122102101F039F810BD44
:107B800008230A001A40194202D14BB2002B0FDA27
:107B9000102101F02DF8002808D02300F2331B78C3
:107BA000002BECD0F1342378012BE8D10020E6E75C
:107BB00003208907FAD4E2E7F0B51F00184B85B01F
:107BC0001C68019002910392002C27D1200005B07F
:107BD000F0BDA5683301ED186B89019A934211D36A
:107BE000029A93420ED8002F04D10A9B002B10D189
:107BF0002C00EBE73B002978039A6868FEF7F6FC57
:107C00000028F2D10136B6B2A388B342E1D8246885
:107C1000DAE7A3680A9A5B891380E9E70026F3E7AD
:107C20001465FF1F37B50C000A884988012391426B
:107C300017D3002A15D0651D23792A0002210A488E
:107C4000FEF7D4FC102300280BD02379618820880C
:107C500000242A000094FFF7AFFF0A23A04200D0BF
:107C6000230018003EBDC046FABF001113B50A003C
:107C700008884988012388420BD8002809D00024AD
:107C8000137905320094FFF797FF0A23A04200D032
:107C90002300180016BD13B50A000888498801237F
:107CA00088420BD8002809D00024137905320094AB
:107CB000FFF782FF0A23A04200D02300180016BD60
:107CC000F0B58BB003904A8808880E0001238242E9
:107CD00055D3002853D00023012704AC2370002281
:107CE000718813000092FFF767FF051E3ED02078D1
:107CF000002835D12B78022B18D167706A89830050
:107D00000130E31880005A8069680222201803F0CD
:107D100083FD23780133DBB22370042B19D93B0098
:107D20006889013080B2002BD9D01FE00223637034
:107D3000122358436A89231804305A806968102234
:107D4000201803F069FD23780133DBB22370002B88
:107D5000E5D10C4A6B899B185A425341DBB2DFE7ED
:107D60006378012BE4D12B78022BC7D022780A2329
:107D7000002A04D021000398FEF798F90023180088
:107D80000BB0F0BD0100FFFF0F4BF0B50400186809
:107D9000002816D083685D89A54207D88288AE186E
:107DA000B44203DA12019A18934201D10068EFE756
:107DB0001E005F891036A74204D1002900D00D8033
:107DC0001800F0BD3300EFE71465FF1F70B5050024
:107DD0000C0008880021FFF7D7FF03000120002BCB
:107DE00004D022002800197AFFF7C1FE70BDF7B554
:107DF0000C00002501902300EE331B78AB4201D824
:107E000000200AE06B00E65A00213000E718FFF777
:107E1000BBFF002802D126800130FEBD017A019807
:107E2000FFF794FE002802D03B882380F5E7013558
:107E3000EDB2E0E710B5040008880021FFF7A4FFC9
:107E400003000120002B03D02000197AFFF77EFEEB
:107E500010BD0000054B1B68002B01D1180004E089
:107E60009A6852898242F6D1988870471465FF1F3C
:107E7000F0B50E27002687B0039302ABFF183E80B3
:107E800005001F4B40891400984207D02B78013021
:107E900000976A6880B2FFF78FFE060002212B78F8
:107EA00018486A68FEF7A2FB00280FD06C892000F2
:107EB000FFF7D0FF002802D0013C0419A4B2039BB5
:107EC000002B00D01C80300007B0F0BD02212B78C1
:107ED0000D486A68FEF78AFB0028E7D102212B785B
:107EE0000A486A68FEF782FB002807D0002EDED021
:107EF0003B88A342DBD17489013CDFE76C89DEE774
:107F0000FFFF0000FABF0011F8BF0011F6BF00111B
:107F100010B50C00FFF7DEFC03000220002B0AD096
:107F2000002C00D023609B781720FE2B03D0013853
:107F3000FF2B00D1002010BD73B50D0001A9040076
:107F40001600FFF7E5FF172805D0002E04D1290001
:107F50002000FEF727F976BD01221021200000F055
:107F600047FE0028F3D0F6E7014B18607047C04683
:107F70002465FF1F37B56B469D1D010004000222DA
:107F8000280003F079FD2B88B02B0ED12379122B1A
:107F900009D12300FA331B78012B06D10121608817
:107FA00000F0E0F801E01B2BF8D037BD10B5054B11
:107FB0000421187000F098F8FFF74CFDFEF770FBF5
:107FC00010BDC0462865FF1F0020F0B50BB20F00A2
:107FD00087B0834234DA274B187803F0FDFD051E85
:107FE0002BD00378A02B25D103AE3100FEF7E4F8A7
:107FF000041E0BD1B378DB0724D51F4B06341B6856
:10800000002B03D03100688898470400A868002836
:1080100001D003F0E1FC002C08D1184A039B134067
:10802000174A934206D0B3781B2B03D001216888EE
:1080300000F098F8280003F087FD802000027840C7
:1080400007B0F0BD0F4B1B68002B10D031006888C3
:108050009847041EDAD07378002BD7D1B27801A9E3
:108060000A704B800C716888FDF7F6FFCEE7062496
:10807000F1E7C0462865FF1F2065FF1F00FFFF00D6
:10808000000112002465FF1FF7B50190FC200D00D0
:1080900017001E0003F0E0FC04001320002C12D097
:1080A000B02320002370089BF4226770658026713E
:1080B0000830002B08D0190003F0AEFB2100019816
:1080C00003F082FB0020FEBD089903F00DFEF5E7EA
:1080D00010B5041E06D00078FD2803D803F094FCE8
:1080E000FF23237010BD00000A1F93B210B50400D7
:1080F0000220032B05D882400020024BD1529B184E
:108100009C7010BD4865FF1F0B8870B5043B0400D0
:108110000D000220032B0BD80121200000F04CFDA4
:1081200003001420002B03D02900200000F0DEFB08
:1081300070BD000007B51300034A00920A00012138
:1081400000F02CFC0EBDC0467183001107B50192F2
:1081500003220092024B0A00122100F049FC0EBDDE
:10816000EF83001107B56B4601AA11800449D8803E
:1081700008780633012802D1190003F00DFB07BD72
:108180002965FF1F0C4B10B518700023FF210B4A07
:108190001380138193819380094A53801370517225
:1081A00093819372D174D3821375517703F03CFBA2
:1081B00000F0FCF910BDC0465865FF1F4865FF1F61
:1081C0002A65FF1FF0B58DB06B46002003910C228D
:1081D0009B5E834200DBB0E05D4B187803F0FCFC53
:1081E000051E00D1A4E00378902B00D09DE006AFDF
:1081F00001004688380000F013FA7968040000296D
:1082000000D19CE03B88052B6ED13B89032B1CD908
:1082100005AC200000F0A2F86288172A61D83989DD
:10822000131D994231D17968237804310291D9071D
:1082300038D5607800F08EF9071E06D00023037150
:108240002378012B08D0132B23D0A868002800D155
:1082500078E003F0C1FB75E06288029909A800F09C
:10826000A6F80290380000F08BF909AA2378387A32
:108270000192002231000092029A00F012F93800B7
:1082800000F064F9029B002BDFD0300000F080F991
:10829000DBE70378032BD8D16288029909A800F0A4
:1082A000D6F8DEE7122B13D1029909A800F0B5F831
:1082B000021EEAD127498B88002BC6D0887909A9EC
:1082C0002378019161780091310000F0EAF8BCE771
:1082D000002302AA93833000617809AAFFF72AFFDE
:1082E000B3E71D4B0993F6E7042B02D09A1F012A2E
:1082F000ABD8184A043B9B00995A0029A5D0D21844
:10830000907831003A0000F0AEF800289DD13B880B
:10831000042B03D001213000FFF724FF012C04D1EE
:10832000A868002801D003F057FB280003F00CFCDC
:108330008020039B0002434018000DB0F0BD0128CF
:1083400000D182E701213000FFF70CFFEDE7C046C6
:108350005865FF1F4865FF1F010017000B78037069
:108360004B784370CB788A781B0213434380704765
:108370000A88030002700A88120A42700A88012AD9
:1083800006D14A8882704A88120AC2700420704757
:1083900002208242FBD14A8804309A704A88120A2D
:1083A000DA708A881A718A88120A5A71EFE710B552
:1083B0000400012082420CD94B780A781B02134337
:1083C0002380834206D1CB788A781B0213436380D3
:1083D000002010BD022BFBD1CB788A781B021343FF
:1083E00063804B790A791B021343A380F0E70B8863
:1083F00003700B881B0A43704B8883704B881B0AE1
:10840000C3708B8803718B881B0A4371CB8883717F
:10841000CB881B0AC3710820704703000120082A7B
:1084200014D14A780878120202431A80CA788878F0
:10843000120202435A804A790879120202439A8052
:10844000CA798879120202430020DA80704710B599
:1084500004000120022A05D100204B780A781B0273
:108460001343238010BDF8B5060010200F0015003F
:1084700003F0F2FA04000120002C0ED0A0230C22FD
:10848000290023806780201D002D07D003F0C4F948
:108490002100300003F098F90020F8BD03F024FC1F
:1084A000F6E7F7B51E00009008AB142017001D7802
:1084B000019103F0D1FA041E12D0A2230370019B94
:1084C00047704380099B057146710C220830002BD0
:1084D00007D0190003F0A0F92100009803F074F907
:1084E000F7BD099903F000FCF6E737B5041E0FD07D
:1084F0004388002B0CD00025C1881323007A172253
:1085000001950095FFF7CDFFFF236580637225700D
:1085100037BD000010B50C4904004A88002A09D074
:108520008B89002B05D00020CB8A0222834201D008
:1085300010BD012213000A20434300204032C854DA
:10854000C81842800472F3E72A65FF1F00234380A6
:1085500003707047094B00211A0010B55C88002C8D
:1085600006D01C79844203D10A234B43D01810BD96
:1085700001310A330329F1D10020F8E72A65FF1FF2
:1085800010B50400407A03F03FFAFF23637210BD78
:108590007047043010B580B203F046FB002803D0CA
:1085A0000421494203F078FA10BD000070B500259F
:1085B000104CA0682580A581A580A84202D003F0B8
:1085C0000BFAA56000250C4C0C4B606D1D80230040
:1085D00058331D70A84202D003F0FEF965650025EE
:1085E0006068002801D003F0F7F9013508340A2D3E
:1085F000F6D170BDF065FF1F9465FF1FE465FF1F96
:1086000070B5041E09D1054D2880A881A880A868EE
:10861000002802D003F0E0F9AC6070BDF065FF1FE8
:10862000F0B54B8885B00193002343600A790500BB
:108630000F00022A00D07BE0CA88032A17D98B6872
:108640005E7819783602DC78D8790E4399781B7AEF
:1086500024021B020C43034353495BBA0B80331DB6
:1086600093421ED1042C04D0631F022B0ED901208B
:1086700015E0019A4D4B1201D35A002B06D00198F8
:10868000FFF7BEFF4A4A1369013313610421B8683A
:108690002E812C80494203F0FFF96860002005B06C
:1086A000F0BD434D042C06D0631F022B0FD9EB689D
:1086B0000133EB60DBE7019A3C4B1201D35A002BEC
:1086C00005D00198FFF79CFF2B6901332B61374BD5
:1086D00030000293019B029A1B0101930023019930
:1086E0008C468B52130063449C8003939E81FFF75A
:1086F00050FF039B041E986016D00421B8684942BD
:1087000003F0CAF9FA880100043A200003F084F863
:108710000199029AFB888A5A043B9B18029A8B5251
:108720002B6801332B60A2E7AB690133AB619EE795
:108730001E4B0293019B1E01029BF35A002B2DD06E
:1087400002998C19A068002828D0012A26D1FA881D
:108750009B189BB27352A189994217D39B1AC018D8
:10876000B96803F059F8029BA289F35A934200D0EA
:108770007DE700222B81A3882B80A3686B60029B7E
:10878000F2520B4A53680133536070E7084A93680A
:10879000013393600198FFF733FF68E7044A536998
:1087A00001335361F6E7C0465A65FF1FF065FF1FAE
:1087B0006065FF1F70B5051E15D10B4C0B4B188063
:1087C000230058331870606D002802D003F004F9BC
:1087D0006565250050356068002801D003F0FCF87D
:1087E0000834AC42F7D170BD9465FF1FE465FF1FEC
:1087F000F0B51700A12285B0920001934243394B96
:1088000006001B680C009B18D933FF331D78FDF759
:1088100041FF0430854204DD3000FDF73BFF0430AA
:10882000C5B2BD4207D33A0000213000019B03F0DE
:108830008BF805B0F0BD2900380003F08DFA230055
:10884000C6B250331E700393019B29006365380044
:1088500003F05AF9CBB20293002B02D0039B0136EE
:108860001E7000262300503303931B78B34204D8B4
:10887000606D002831D10020DBE7029A2800002A31
:1088800004D0013B1000B34200D02800F700E719E4
:10889000387003F019FA786000280ED03A78019900
:1088A00002F0BAFF019A3B780136D3180E4A0193C1
:1088B000D369F6B20133D361D4E7039B18706065C6
:1088C000A74205D1084A1320D36A0133D362B0E727
:1088D000606803F081F80834F2E703F07DF80023C4
:1088E0006365C8E73409FF1F6065FF1FF7B50D001A
:1088F00007000421686803F0CFF82B890400037097
:108900002B891B0A43702B8883702B881B0AC3702A
:108910002E8902250436F6B2F42E15D81B4B9F4241
:1089200014D10C2003F098F81135011E0CD09023BF
:1089300003708E3B0371043B4380154B8460C680FB
:10894000187802F041FF00252800FEBD5C237B4320
:10895000104AD3180093583301931B78002B0FD182
:108960000300320038000099FFF742FF019B050029
:108970001B78002BE8D13800009902F015FFE3E7DF
:10898000054A0725536A01335362DDE7FEFF000005
:108990005865FF1F9465FF1F6065FF1FF0B587B026
:1089A000009017200F0016000193FFF7F2FD13252A
:1089B000041E19D00C98031E02D00199201D98475F
:1089C000030AE370052302AAA07004309081277087
:1089D0000098667003A993800494FFF787FF051E33
:1089E00002D0200002F0F8FF280007B0F0BD000020
:1089F000F0B587B01F000CAB1B78039105930121E4
:108A00000DAB06001C78049200F0D6F8142500285F
:108A100021D02000FFF77EFD0135041E1BD0114937
:108A2000059B0A7803700132D2B2131EC68001D1B1
:108A300001231A000B7022713000049B03990097E8
:108A4000FFF7ACFF051E09D1230021000648074AA5
:108A5000093303F099F9280007B0F0BD00236380C3
:108A60002370F8E75C65FF1FEB8400113075000090
:108A7000F8B505000E00064C064F2368002B02D007
:108A80003100280098470434BC42F6D1F8BDC046F6
:108A90000066FF1F1466FF1F0123064A5B425380D6
:108AA000002313715362044A136053609360D360D0
:108AB000136170471466FF1F0066FF1F020000234A
:108AC00010B506499C000859002801D1625010BD1C
:108AD0000133052BF6D11320F9E7C0460066FF1FCE
:108AE000034A5388181A4342584140421040704785
:108AF0001466FF1FF0B585B002930AAB1F780CAB6C
:108B00001B88009008000E0001920393FFF7E8FF16
:108B100005001120002D1BD10E48FFF7E1FF0400D6
:108B20001520002C14D006220B99A771E01D02F02D
:108B300073FE019B30002371029B29006371009B2F
:108B400066802370039B6562E381FFF791FF280035
:108B500005B0F0BDFFFF000010B5FFF7C1FF040036
:108B60000220002C12D060880121FFF781FF606A8B
:108B7000002801D003F080F828220021200003F013
:108B8000B3F8012300205B426380207110BD000018
:108B900030B5074A074C5588010013780020A542DC
:108BA00004D05B1A59424B415842104030BDC04678
:108BB0001466FF1FFFFF0000084A10B501230C00D8
:108BC000904208D0FFF78CFF031E04D003792340A6
:108BD0005A1E9341DBB2180010BDC046FEFF0000D4
:108BE000024B1879431E9841C0B270471466FF1FAC
:108BF00070B504000D001600FFF772FF002804D1C5
:108C00000D4B9C4200D0143070BD416A03790520A1
:108C1000002907D012221A40102A02D10520002E66
:108C2000F2D10F20DB06EFD5897E0C20A9428941C5
:108C3000494249420840E7E7FEFF0000030010B543
:108C4000002800D110BD0348034A41889142F9D061
:108C50009847F7E71466FF1FFFFF0000002330B5B9
:108C6000C45CCD5C6C40D4540133102BF8D130BDC2
:108C70000F23002210B5C45C64002243CA54C25CB6
:108C8000D209013BF7D210BD0200010010B520321D
:108C9000103102F021FF10BDF0B58BB00390102011
:108CA00005931700049102F057FF0090102002F086
:108CB00053FF009B13240190002B05D000280CD1FA
:108CC0001324009802F0D8FF019B002B02D018005B
:108CD00002F0D2FF20000BB0F0BD102002F03CFFEC
:108CE0000600102002F038FF13240500002E00D1EA
:108CF000AEE0002819D01022002102F0F5FF32006A
:108D00002900039802F0E8FE041E0ED133787F2B71
:108D100051D830000099FFF7ABFF009B1B787F2BE9
:108D200053D801990098FFF7A3FF300002F0A4FF89
:108D3000002D02D0280002F09FFF002CC1D110208E
:108D400002F00AFF0600102002F006FF0290002E3B
:108D50007CD0002878D03A000F3223000125121170
:108D600005D00F333B4015B25A4253411BB26A1E25
:108D70001201002B33D0049BD2B298180099029AAA
:108D8000FFF76CFF013D10220021300002F0ACFF24
:108D9000ADB2049F2D017D19AF4242D0002C33D0DB
:108DA000300002F069FF029B002B00D189E7180018
:108DB00002F062FF85E729003000FFF759FF280025
:108DC0002549009AFFF74AFFA7E729000098FFF717
:108DD0004FFF28002049019AFFF740FFA5E70F2128
:108DE0000F4004998A18D9B28F4208D9D15C06A8DD
:108DF00019540133102BF6D1029A0199C0E7791A60
:108E000048424141C901F2E73900300006AAFFF7A4
:108E100025FF3200039806A902F05EFE1037040019
:108E2000BAE7002CBCD13000029906AAFFF716FF62
:108E3000320006A9039802F04FFE08220400310018
:108E4000059802F0E9FCABE71324A9E71324AAE78D
:108E5000002800D06EE733E700C00011F0B58BB0FA
:108E60000F0016000225009000283FD0002A3DD0B8
:108E70000B1DDBB21800029302F06EFE1135041ECA
:108E800034D0FDF747FD05003A000099201D02F09F
:108E900083FEEBB20393E3702B0CDBB22F0A00933B
:108EA0006370FFB22B0E2370A7700193FDF72CFDAA
:108EB0001022010006A802F06FFE2100029A04AB06
:108EC00006A8FFF7E9FE051E0DD1039B08223370AB
:108ED000009B04A9B370019B7770F370301D02F002
:108EE0005BFEFDF71DFD200002F0C6FE28000BB062
:108EF000F0BDF0B58FB00D00149E03900492059361
:108F0000002A03D1022420000FB0F0BD002EF9D0BA
:108F10000398FFF7E5FD1424071EF4D07278337828
:108F200012021A43B3781B041343F27812061A4351
:108F3000036A0192934201D30133E3D1002D03D0A0
:108F40003B7901249B07DED50822002106A802F008
:108F5000CBFE059B13240433DBB21800029302F00E
:108F6000FBFD051ECFD0059A0499043002F014FED3
:108F700004223100280002F00FFE390010221031C7
:108F80000AA802F009FE2900029A06AB0AA8FFF718
:108F900083FE041E0FD1082206A908A802F0FCFDDA
:108FA0000822311D08A802F05FFC012807D10199B1
:108FB0000398FDF7C9FC280002F05EFEA3E7012438
:108FC000F9E7000070B51C4C05002368181E10D08E
:108FD000002D14D11A78002A0CD1981C083202F006
:108FE0001BFC02F009FC0135002808D123681D7024
:108FF000012070BD0A331800082202F00DFC23681E
:10900000002BF5D0122002F027FD061E0DD0C12343
:1090100021680370457002311022023002F0FCFB1F
:1090200023683100587802F0CFFB206802F024FE5C
:1090300000232360DCE7C0463C66FF1FF8B5040050
:109040002020FDF755FB0D4EA700BB590500002B56
:109050000DD000280BD0D878FF2809D108492A0064
:109060000C55F35907480333611802F08DFEF8BD23
:10907000290002F001FC0028F0D1F8E75866FF1F34
:109080004066FF1F95A2001170B5064D840063591C
:10909000002B05D0D87802F0B7FCFF226359DA70B4
:1090A00070BDC0465866FF1F70B506008CB00C003E
:1090B000150000213022684602F016FE3100102211
:1090C000684602F069FD1D2021000322684402F079
:1090D00063FD6846FFF7D8FD2D2104000322280018
:1090E000694402F059FD20000CB070BDF0B50700D6
:1090F000160097B001931CAB1D7830221EAB009177
:109100000AA800211C7802F0EFFD102239000AA8FD
:1091100002F042FD1022002102A802F0E5FD072224
:10912000310002A802F038FD072202AB9818631E36
:109130009C41019902F030FD02AB9C732B005A1E3A
:10914000934102AAD3730021102206A802F0CCFD9D
:1091500006221D9907A802F01FFD1A2002ABC018B5
:1091600006221F9902F018FD102200990EA802F0A5
:1091700013FD102202AB0EA908781C78013A60405A
:10918000D2B2087001330131002AF5D10AA8FFF7E5
:109190007BFD102212A904000EA802F03DFB102254
:1091A00006AB0EA908781D78013A6840D2B2087063
:1091B00001330131002AF5D10AA8FFF765FD044308
:1091C00010222098E4B212A902F0E6FC200017B0A9
:1091D000F0BD70B50E0014008CB00100102268467E
:1091E0001D0002F0D9FC3100082204A802F0D4FCD2
:1091F0002100082206A802F0CFFC6846FFF744FDD4
:1092000004001022280008A902F0C6FC20000CB0BF
:1092100070BDF8B506000D0000243719AC4200D32C
:10922000F8BD02F0A1FA030A3B70631CDBB2013700
:109230009D4203D90234F054E4B2EEE71C00EDE79E
:1092400073B506000C000225002819D0002917D09C
:10925000032101A8FFF7DDFF6B469A793F231A40EF
:10926000013313436A463000937101A92200FFF7CE
:109270001BFF051E04D10322E01C01A902F0CCFA59
:10928000280076BD03785807DA08C00FD2008000A6
:109290009B0710439B0F1843C0B2704707230B4036
:1092A000C908C9000B4303707047000070B5040083
:1092B000FFF7EAFE134DA4006359002B21D0186A72
:1092C000002801D002F0D8FC2B59986E002801D05C
:1092D00002F0D2FC2B59D86E002801D002F0CCFC51
:1092E0002B59186F002801D002F0C6FC2B59586F7B
:1092F000002801D002F0C0FC285902F0BDFC002378
:109300002B5170BD5866FF1F0E4B8000C35870B5BF
:109310000C00002B0FD09D68002D0CD02B78201D49
:109320000B706B784B70A97CFFF7B8FF2B7E237214
:109330006B69E36070BD10220021200002F0D4FCB4
:10934000F8E7C0465866FF1F014B18607047C046DB
:109350005466FF1F074A03008000825810B5002A98
:1093600006D0D088984203D1012901D1FFF79EFF92
:1093700010BDC0465866FF1FF0B5264E95B0870059
:109380000B93BB590500099112200A92002B31D092
:10939000D888FFF7A5FB04001420002C2AD0280051
:1093A00010A9FFF7B1FFBB591E781D6A002E23D00C
:1093B0000895FDF7EFFA07000020FDF7F1FA079096
:1093C000A379E61D069310AD0CA9089800F0E2FA07
:1093D0000EA9280000F0D7FA0B9B0A990493069B6C
:1093E00009980293079B0396019300970EAB0CAA72
:1093F000FFF77CFE15B0F0BDFDF7CCFA069030000B
:10940000FDF7CEFAE31DA779079310AB060008938A
:10941000DAE7C0465866FF1F30B50C4C85002A5964
:10942000030085B00120002A0ED018006946FFF71E
:109430006BFF2B591A78D888054B002A00D1054BB1
:109440006A46072100F0D9FB05B030BD5866FF1F02
:10945000879900119599001130B5094C850029595B
:1094600085B010226846253102F0D6F92A5911211B
:10947000044BD0886A4600F0C0FB05B030BDC04642
:109480005866FF1F319A001130B5094C85002959E3
:1094900085B010226846353102F0BEF92A591121F3
:1094A000044BD0886A4600F0A8FB05B030BDC0462A
:1094B0005866FF1F6F9A0011F7B54D4F86001020B8
:1094C000F4590D0002F048FBF3592062186A132288
:1094D00000286CD0033A29009C6802F09DF9F359EA
:1094E0001A780192002A58D11E6A227D317B944657
:1094F00051400122019F114201D167461740217D51
:10950000914339432175377B4F40BC466046002765
:10951000800701D44F081740012102208F40227D8F
:1095200082433A432275377B5740BC46604600274A
:10953000400701D497080F400420227DBF008243DA
:109540003A432275627D002794466046727B424012
:109550000A4201D167460F400121627D8A433A43A6
:109560006275777B5740BC4660460027800701D470
:1095700057080F400220627D7F00824317436775C2
:10958000767B00227E40760701D4BA080A40042682
:10959000617D9200B1430A4362756A78002A08D05F
:1095A0006278002A05D005220533DA770022100000
:1095B000FEBD04222979114205D1A17C114202D1BC
:1095C0000533033AF1E7019A21782C78002A02D179
:1095D0000A002100140018220429E8D8042CE6D837
:1095E00005206043034A05331218525CDDE7C0468C
:1095F0005866FF1F10C0001110B50A001121024B60
:1096000000F0FBFA10BDC046CB9A00110B0030B53C
:1096100087B001AD2B806B4604001100981D082215
:1096200002F0FAF82A000B212000024B00F0E5FAC4
:1096300007B030BDF39A001110B50A001121024B9A
:1096400000F0DBFA10BDC046479B001113B50B00BC
:1096500011006A4613706B4604000622581C02F083
:10966000DBF86A4608212000014B00F0C6FA13BD62
:10967000679B001110B50A001121024B00F0BDFAE2
:1096800010BDC046B79B00117FB505000B4BAA006B
:10969000D4580800002C0FD0666F237FE288217811
:1096A0000396266F0296E66E0196A46E0094FDF76F
:1096B00009FC2800FFF7FAFD7FBDC0465866FF1F72
:1096C00010B51721FFF7E0FF10BD000070B50A00CC
:1096D0000D00064B0221040000F08FFA06002978E5
:1096E0002000FFF7D1FF300070BDC046979A0011EF
:1096F00070B586B000236A461370836804001D7835
:10970000681E0A2859D801A902F036F9060633372F
:109710003B3F43474B4F5300180000F042F90623EC
:1097200012284BD000281BD16088FFF7D9F90823F5
:10973000002813D04279002A47D1264B1A780723F4
:1097400012070BD5244B1A680723002A06D0166887
:10975000002E03D0290001AAB04703006A46137007
:109760006B461B786088002B2AD1FFF767FC06B098
:1097700070BD180000F06CF9D4E7180000F087F90C
:10978000D0E7180000F093F9CCE7180000F0ADF92D
:10979000C8E7180000F0C3F9C4E7180000F0F6F9B4
:1097A000C0E7180000F0F6F9BCE7180000F013FA63
:1097B000B8E7180000F013FAB4E707236A461370FD
:1097C00069466088FFF782FFD1E70523012AC5D1EA
:1097D000024BB8E7E564FF1F5066FF1F5466FF1F8A
:1097E000F8B52C4F8600F35904000D00002B40D033
:1097F000DA8882423DD15A78062A33D11A78002A73
:109800002ED0012099681A6A097D014206D0157B85
:10981000054203D007225A700120F8BD0220014200
:1098200004D0157B054201D00922F4E7042001424F
:1098300004D0127B024201D00B22ECE7164B1B68CE
:10984000002BE9D05B68002BE6D020009847BB597D
:1098500000215B78122BDFD12000FFF715FFDBE73B
:109860000E4BECE7112A04D1002900D03225290043
:10987000F2E7002D08D12000FFF732F9002803D0CD
:10988000102302791343037121002800FDF798FA91
:10989000C2E7C0465866FF1F5066FF1F5466FF1F91
:1098A00070B50E4E8500AB590400002B13D01B7809
:1098B000002B11D10A4B1B68002B04D05B68002BD6
:1098C00001D02000984773595B78122B03D10021F7
:1098D0002000FFF7D9FE70BD024BECE75866FF1F72
:1098E0005466FF1F5066FF1F094B8000C3581020AD
:1098F000002B0CD01A6A002A09D09B68002B06D0D6
:10990000127A1B7E101C9A4200D9181CC0B27047F4
:109910005866FF1F70B503000D0014000220002AD6
:1099200030D000292ED013700B78081D53704B785F
:109930009370FFF7A7FCE070012002212B7A2371BE
:109940006B7B034063716A7B0A401343042263719B
:109950006E7B1640334363716E7BF608F60033432B
:1099600063712B7B0340A371287B014000200B43D4
:10997000A371297B0A401343A3712A7BD208D2002A
:109980001343A37170BD10B50A0001000120FFF759
:10999000C1FF10BD10B50A0001000220FFF7BAFF99
:1099A00010BD70B506000C000220002E30D000293A
:1099B0002ED07378201D0B70B3784B70F178FFF7C1
:1099C0006DFC01223579257271794B100800134026
:1099D000934010400343881010408000C90803439F
:1099E000C9000B436373B1794B10080013409340D7
:1099F00010400343881002409200C9081343C90075
:109A00000B4321202373FCF773FE854201D2122001
:109A100070BD2220257AFCF76BFE8542F7D82378AB
:109A20001820042BF4D86378012BF1D80020EFE73D
:109A3000030010B50220002909D0002B07D0032213
:109A4000481C0A7019000D3201F0E6FE002010BD1E
:109A500003000222080010B5002B06D0002904D014
:109A60000E32591C01F0D8FE0022100010BD030078
:109A700010B50220002909D0002B07D00422481C71
:109A80000A7019000C3201F0C7FE002010BD10B59D
:109A9000FFF7DEFF10BD03000220002906D0002BD7
:109AA00004D0052200200A701B784B707047030019
:109AB0000220002B08D0002906D05B7800200B7014
:109AC000013B082B00D918307047030010B5022065
:109AD000002909D0002B07D00622481C0A70190063
:109AE0000A3201F099FE002010BD10B5FFF7B0FF5B
:109AF00010BD02000B00022010B500290ED0002A74
:109B00000CD007211970118859701188090A9970B1
:109B100011180822D81C01F07FFE002010BD0300A0
:109B20000A00022010B5002B0CD000290AD0997829
:109B30005878090201431180901CD91C082201F0B9
:109B40006BFE002010BD030010B50220002909D0D3
:109B5000002B07D00822481C0A701900921801F047
:109B60005BFE002010BD02000B00022010B5002992
:109B70000BD0002A09D009211970117818185970D2
:109B8000511C062201F048FE002010BD10B5FFF761
:109B90005FFF10BD02000B00022010B5002A09D0A3
:109BA000002907D05178197011180622581C01F0AD
:109BB00033FE002010BD030010B50220002909D09B
:109BC000002B07D00A22481C0A701900063201F047
:109BD00023FE002010BD10B5FFF73AFF10BD0200B4
:109BE0000B00022010B5002A06D0002904D018006E
:109BF0005178FFF753FB002010BDF0B585B017007A
:109C00001E006A4606230500080091819380FEF736
:109C1000C0FC1324011E02900CD03800B047041E73
:109C200005D1280001A9FEF76FFA041E02D00298A0
:109C300001F0D2FE2800FFF701FA200005B0F0BDC8
:109C4000F0B504008BB0019115000021102202A88C
:109C500002F04AF8334EA700B85900283CD0C38818
:109C6000A34239D10378002B36D14278062A18D185
:109C700002000100553235310C3006ABFFF7A9FA6E
:109C8000002829D12000FFF72FFE020006A902A814
:109C900001F0C2FD200002A901F0DEFF01200BB09F
:109CA000F0BD816E002917D00B8A112A28D19D4260
:109CB0000ED101981231093A01F0D6FD012807D1E1
:109CC000BB5920009D6EFFF70FFE29000200DEE762
:109CD00032212000FFF7D8FC2000FEF701FF061E0E
:109CE0001BD0416A002918D00B8AAB4215D108223B
:109CF0000198123101F0B8FD01280ED1716A0AE015
:109D00009D42E9D108220198123101F0ADFD0128F0
:109D1000E2D1BB59996E8A7EB9E7200001F094FF29
:109D2000BCE7C0465866FF1FF0B56B4D87007E59F3
:109D300085B0337802900393002B00D087E0B3689E
:109D4000346A01937078062817D101221B7D1342D3
:109D500002D0217B114218D10222134202D0217B72
:109D6000114251D10422134203D0237B134200D06D
:109D70008BE0019B5A7DEB5991E007380428F8D815
:109D800001F0FAFD032E42678300B36E002B03D16E
:109D90001C2001F0E1FEB066EB599C6E002C1CD03B
:109DA00010220021200001F09FFF0298FFF79CFD88
:109DB00001002000FFF72DFA01F0D6FC20822000E0
:109DC00008211230FFF725FA0298FFF78DFDA076E3
:109DD000EB592100D888FFF70FFC0822EB591CE053
:109DE000B36E002B05D01A00198AF0881232FFF7E3
:109DF0000DFC0222019B197DEB5911423DD0207BC5
:109E000010423AD0073208E0F488FCF7DBFD01008D
:109E10002000FFF711FC0A22EB595A70029B9C00AC
:109E20002A595378073B042B11D8D088FEF758FEE7
:109E300000284ED0C3895A08D2182849029B02989C
:109E4000CB542B5941180433254801F09DFF05B030
:109E5000F0BDFCF79FFD03000120834201D10020EB
:109E60000393EB59DE88FCF79BFD03990200300059
:109E7000FFF7ECFB019AEB59117D042211420CD043
:109E8000217B114209D00B22C7E7F688FCF73CFD85
:109E900001003000FFF7EEFB6BE7019A527D0121D4
:109EA0000A4204D0607B084201D00C22B5E70221AF
:109EB0000A4204D0607B084201D00E22ADE70421A3
:109EC0000A4204D0627B0A4201D01022A5E7122286
:109ED000A3E7FA225200B0E75866FF1F5C66FF1F37
:109EE0009FA2001110B5064B1A78042310001840E9
:109EF0001A4200D00348FFF727FA002010BDC046E1
:109F0000E564FF1F8443FF1F70B50400FFF7D4FA18
:109F1000051E43D12000FFF77FFA234EA400A0596D
:109F20008268937CDB0708D50321036A1B790B4009
:109F3000012B02D1017F0B430377431DD97F8B1E79
:109F4000022B0DD8022900D00121C088FCF790FF18
:109F5000042133591A7F59700A431A77280070BDBB
:109F600001290CD102231022437000210C3001F092
:109F7000BBFE305910213530FFF74BF9EEE70529CC
:109F8000ECD10223D118437010220C3001F044FCB4
:109F900004233259117F0B431377EAE70825182869
:109FA000DCD1053DDAE7C0465866FF1FF0B58BB03F
:109FB000059143887E4F9E00F45915000493002CB0
:109FC00015D1012902D000200BB0F0BD101D57782B
:109FD0001678FFF757F9EB68320002932B7A049951
:109FE000019300903B002000FCF70CFFEBE7E388B7
:109FF000049A934201D00820E6E72378012B00D190
:10A00000D4E0059B581E092800D9CFE001F0B4FC2C
:10A0100005CE0A29CC506C859AB229000498FFF726
:10A0200073FFD1E7200029001022453001F0F4FB36
:10A03000B9594B78042B02D1013B4B70C3E70B009D
:10A040000A00253335320C310498FFF795F904984E
:10A05000FFF702FA0522431E9841BB59C0005A700F
:10A06000B2E7200029001022553001F0D5FB049BF7
:10A070004F4C9D00295904980A0006AB55320C310B
:10A08000FFF77AF929591022453106A801F0ECFBB7
:10A09000012808D10498FFF7F7F90590002804D1AA
:10A0A00006222B595A7005988EE708230593FAE784
:10A0B00063780C2B7AD1E36E002B03D11C2001F0C6
:10A0C0004BFDE066BB59D86E00286FD010222900E6
:10A0D00001F0A2FBBB590498DC6EFFF705FC0D22D2
:10A0E000A076BB595A706EE7E06E00285ED06378A8
:10A0F0000D2B5BD12B8808220382A91C123001F0A2
:10A100008BFBBB599A68517D0222114226D0186AF6
:10A11000407B104222D00C32E4E763780E2B45D10D
:10A12000236F002B03D1162001F016FD2067BB59C9
:10A13000186F002803D01022290001F06DFB0F22B8
:10A14000BB59CFE763780F2B30D1206F0622691CF3
:10A15000103001F061FBBB599A68517D0422114215
:10A1600003D0196A497B1142D5D100210498FFF729
:10A170008BFA28E7636F002B0DD0BB59586F00286E
:10A18000F3D01022290001F047FB0122BB595242B3
:10A190005B6F1A61E9E7142001F0DEFCBB596067D0
:10A1A0005B6F002BE9D126E72978DFE707200BE773
:10A1B0005866FF1F10B5064C207001F0F5FB062114
:10A1C0002078FDF791FF0348FEF778FC10BDC046EC
:10A1D0006B66FF1F5593001100200BB270B50D0088
:10A1E000834216DA264B187801F0F6FC041E0DD0D7
:10A1F0000378922B0ED0A02B37D0224B1878FF2853
:10A200003AD0210001F0E0FA002835D18020000288
:10A21000684070BD43780E2B0BD03E2BEDD1837878
:10A22000052B12D0082BE8D181798088FFF7D8FA66
:10A2300008E0154B82889A42DFD183681878591C50
:10A24000FEF7C0FE002817D1D7E7104B1B785B073D
:10A2500012D50F4B1B68002B0ED09B68002B0BD028
:10A26000C289811D80889847ECE7FFF741FAA06812
:10A27000002801D001F0B0FB200001F065FCC5E72B
:10A280006B66FF1F7D43FF1F18200000E564FF1F62
:10A290005466FF1F10B50078FFF712FA10BD10B515
:10A2A0000078FFF7FDFA10BD0C234343084A10B5B0
:10A2B0009B185A68002A03D0012901D1904710BD8C
:10A2C0009B68002BFBD00029F9D19847F7E7C046DF
:10A2D0008866FF1F01238340094A10B5946B1C4315
:10A2E0009463506B98435063D46B200098430129CA
:10A2F00001D120001843D063116B0B43136310BDD1
:10A3000000800040F0B500240127154B85B0DA6BC2
:10A31000144E03921A6C0192DA64019BE3403B42B3
:10A3200017D0039DE5403D400295E5B20299280013
:10A33000FFF7BAFF316A736A002908D03900002B91
:10A3400001D0029979402800FFF7C4FF01E0002BFB
:10A35000F9D101340C36172CDFD105B0F0BDC04661
:10A36000008000406C66FF1F064B01215A68C24006
:10A370000A4204D01B68C3401800084070471B6D98
:10A38000F9E7C046008000400122064B82400029C8
:10A3900003D0D9680A43DA607047D9689143D9601D
:10A3A000FAE7C0460038004030B5032444430F4B61
:10A3B000E25C1B199C785D7801232D1B0135AB40B5
:10A3C000013BA340A140DB430C00122807D80849F9
:10A3D00092005218116819402143116030BD054A9E
:10A3E00011680B4023431360F8E7C04657C00011C3
:10A3F00008F0004014F00040C21F70B5D4B206232C
:10A40000092C0BD80125084C9540002908D00021C3
:10A41000FFF7CAFF23682B4323600023180070BD99
:10A420002368AB43F8E7C04600380040214BF0B545
:10A430001B185B78022B21D1032444431E4A1F4E74
:10A44000A35C12199478012215008540B76B013C7A
:10A45000E4B23D43A240B563194C122815D89B00C5
:10A4600000290CD117495B1899680A439A600123A7
:10A47000205C154A834011680B431360F0BD1149FD
:10A480005B18996891439960F1E70E4B00290DD153
:10A4900059690A435A61225C1328E8D00123203A03
:10A4A00093400A49086803430B60E7E75969914301
:10A4B0005961F0E76C66FF1F57C000110080004033
:10A4C0009CC0001100F00040A0F00040A4F000404B
:10A4D000F8B500241B4E1C4D1C4B1B5D012B1FD1DE
:10A4E000194A9269E2401A420BD00122B2569340B7
:10A4F0002200143AD2B2022A09D815494A691343F4
:10A500004B61013402360C35172CE5D1F8BD002221
:10A51000B2560F499200521891680B439360F0E7CE
:10A52000022BEED1E7B23800FFF71EFF012358409F
:10A53000C1B23800FFF77AFF3800FFF715FF6877E0
:10A54000DFE7C04629C000116C66FF1F6D66FF1F64
:10A5500000F00040012202388240054B002903D060
:10A5600059690A435A617047596991435961FAE739
:10A5700000380040F8B50E0001210F008740114A55
:10A580000400D368FD43BB43D360831E8B4201D8D4
:10A59000FFF7E0FF00212000FFF72EFF0A4A0B4BD8
:10A5A0005168012E05D139431B1951605E7000209E
:10A5B000F8BD2940516002221C1962709A69154049
:10A5C0009D61F4E700380040008000406C66FF1F8A
:10A5D000012210B58240074B002906D019680A43B2
:10A5E0001A600121FFF7C6FF10BD19689143196079
:10A5F000F7E7C046008000400C2370B500254343B8
:10A600000A4A29009B181D70094B04001B185D7035
:10A61000FFF7B0FF0123A340064928000A681A4348
:10A620000A6005490A689A430A6070BD8866FF1F80
:10A630006C66FF1F348000403080004070B504001D
:10A640000E00FF2813D003250540FFF7D5FF084A69
:10A65000A3089B009B183F22ED00AA40AE4019685A
:10A6600020009143314319600121FFF78DFE70BD39
:10A6700018380040F8B50C244443134B0500E41887
:10A680006368002B03D1A3681220002B1AD002228A
:10A6900001270E4B00215B195A7028002770FFF725
:10A6A00069FF63681E1E08D0A3683E00002B04D01B
:10A6B0002800FFF759FE4640F6B228003100FFF7A8
:10A6C00009FE0020F8BDC0468866FF1F6C66FF1FAC
:10A6D000F7B5C420FF222B4B80001958002491436A
:10A6E0003F3A0A431A508022274F5202274E1A60DF
:10A6F000274B1D5D002D21D0A31E012B03D8012166
:10A70000E0B2FFF727FF012D18D11F4B9B69E340F3
:10A710002B4213D0E3B218000193FFF725FE01008E
:10A720000198FFF755FFE3B2143B022B1DD801211E
:10A730007156184A8D405369AB4353613B7F002BE0
:10A740000DD0E5B22800FFF795FF2800FFF70CFEBB
:10A750007B7F0100834202D02800FFF7A5FD013472
:10A760000C370236172CC3D1F7BD012100237156D7
:10A77000F3568D40074A9B009B189A68AA439A603B
:10A78000DCE7C04600E100E06C66FF1F29C0001155
:10A790006D66FF1F00F0004070B50E00150004004C
:10A7A000FFF72AFF0C236343094A20009B189D6092
:10A7B0005E60FFF75FFFF021064B074A8900051E28
:10A7C0005A5002D02000FFF717FF280070BDC04686
:10A7D0008866FF1F0000FF1F05A3001170B5134D11
:10A7E00007202C78002C1FD198222100520028002D
:10A7F00001F002FA0123C420FF222B700C4B8000D1
:10A800001C635C630B4B1C605C600B4B19589143E1
:10A810003F3A0A431A50802252021A600D20074A1A
:10A82000074901F059FA200070BDC0466C66FF1F51
:10A8300000800040A0F0004000E100E0D1A600113F
:10A84000D1A40011030010B50620072B09D8054A32
:10A85000137001F089F9D7210020034B034A8900C6
:10A860005A5010BDAC43FF1F0000FF1FCD1BFF1F40
:10A8700070B51D0002240C2910D8094ACA40D2071D
:10A880000CD5FBF741FF041E08D1059A0499280056
:10A89000FBF756FFFCF7C4FDFFF724FB200070BD5B
:10A8A0001210000030B50D7802232C009C43184292
:10A8B00001D02B431C0008252300AB43284201D0C4
:10A8C0002B00234320241D00A543204201D01C431C
:10A8D00025002A230D70184204D011781E3B0B432B
:10A8E000137030BD0028FCD10C2113788B43F7E79F
:10A8F000F8B51D0006AB1B88140007AA0E000B203C
:10A900001778002B27D10A78022A49D14A68507853
:10A9100011780002244A08438018042840D801F026
:10A920002BF803121D1B2300F06801F035F8021C00
:10A93000C0B2B84200D93A1CD2B22000F1682A80D5
:10A9400000F06AFF06E00222F3681B882A80237069
:10A950001B0A63700020F8BD0622EEE701232B805E
:10A96000F3681B782370F5E7F368002B16D00822F4
:10A970002A801A8822701A88120A62705A88A27075
:10A980005A88120AE2709A8822719A88120A6271B1
:10A99000DA88A271DB881B0AE371DBE72B80D9E739
:10A9A00001202B80D7E7C04600D6FFFFF7B5160081
:10A9B0000A781D0008AB1F880C000123022A18D159
:10A9C0004A685078117800022B4A084380180328FF
:10A9D0000FD800F0D1FF02254439E06800F0DCFF19
:10A9E000C0B20723B84204D37B190193152B02DDB3
:10A9F0000D231800FEBDE0682A003100C01900F0E8
:10AA00000BFF6B4600209B88E268D0541B4B1B68F1
:10AA1000834203D01B68834200D098470023E8E7B5
:10AA20000B23002FE5D1022DE2D1737832781B027F
:10AA30001343E2681380114B1B68002BEED01B6898
:10AA4000002BEBD00120E8E70B23002FD1D1062DFE
:10AA5000CED12A003100E06800F0DEFEDEE70B23F5
:10AA6000002FC6D1012DC3D132787533012AC0D849
:10AA7000E3681A70D2E7C04600D6FFFF7868FF1F70
:10AA800070B50C001500072837D800F075FF0414C6
:10AA900036361B36242E182015290BD8184E1622B0
:10AAA0000021300001F020F922002900300000F0E0
:10AAB000B3FE002070BD18200229FBD11288114B73
:10AAC0001A80F6E718200829F4D10A000E48290058
:10AAD00000F0D2FFEDE718200129EBD10B4B1078E5
:10AAE0000B49DA69FFF7DEFEE3E718200129E1D11F
:10AAF000064B10780749DA6BF4E70220DAE7C04624
:10AB00006068FF1F2A44FF1F2044FF1FB043FF1F40
:10AB1000D843FF1FF843FF1F030010B50020DB07D9
:10AB200004D50721024A034800F08CF810BDC04646
:10AB3000B4C00011B043FF1F054A0300106800288D
:10AB400003D082889A4201D1806870470068F6E796
:10AB5000706AFF1F0A88030008009A4204D08A889E
:10AB600004309A4200D0002070470000F8B5F2226D
:10AB700000230D4F0D4E7968050042433370994212
:10AB800000D07B600A4C0021200001F0ADF80023CA
:10AB90001A007C60AB4202D100203370F8BD013353
:10ABA0002280DBB2F234F5E7686BFF1F666BFF1F94
:10ABB000746AFF1F73B56B46019006006846150066
:10ABC0001980FCF75FFF041E11D1002D0FD076898C
:10ABD000002E11D00C2000F0BFFF00280ED0084A34
:10ABE0000460136886808560002B02D1106020000D
:10ABF00076BD1A001B68F7E70224F8E71324F6E78E
:10AC0000706AFF1F012100220A4B10B549420A4C0D
:10AC1000198099809A719A70084B207001201980D0
:10AC20005A60FFF7A3FF2078FCF78AFF0448FDF77E
:10AC300045FF10BD8068FF1F706BFF1F686BFF1F13
:10AC4000F1AC0011022310B5002802D0FFF7B2FFCB
:10AC50000300180010BD0000030010B50020DB0742
:10AC600004D50421024A0348FFF7A4FF10BDC046E3
:10AC7000C8C000113044FF1FF0B50E2687B0039303
:10AC80000CAB1F8802ABF6180500080031000292D9
:10AC9000FDF77AF804000120002C0FD03088FFF770
:10ACA0004BFF03000E20002B08D05E68002E05D05D
:10ACB00021002800039B029A0097B04707B0F0BD1F
:10ACC0000A4B10B5984207D10122002352420A8054
:10ACD0008B708A808B7110BDFFF73CFF0028FAD083
:10ACE00001235B42038000238370F4E7FFFF000031
:10ACF000F8B5050001290AD1134E00243388F22744
:10AD0000AB4219D028001149FFF7DAFF06E002290B
:10AD100004D10139FDF750FF0028EDD0F8BD3B000C
:10AD200063437268D018D35A002B09D03A0000212F
:10AD300000F0DAFF0134E4B2054B1B78A342EED8F1
:10AD400001235B423380DDE7686BFF1F8068FF1FD4
:10AD5000666BFF1F10B5FFF7FDFE03000020834266
:10AD600000D0987810BD0000F0B589B01C000EAB83
:10AD700080CB03901E8810AB1B78049202930B7A51
:10AD80000D00DB0616D42B780593022B24D00498F3
:10AD9000FFF7D2FE002812D003689C46002B0ED08D
:10ADA000029B2200019329003B0064460398009611
:10ADB000A04705E00498FFF7BFFE002802D10E204F
:10ADC00009B0F0BD8368002BF9D00A22290003984E
:10ADD00098470028D7D0F3E76B6858781A786B4B00
:10ADE000000210439842D2D8043B984210D2684BDC
:10ADF000984242D015D8674BC0180128C7D80B20FD
:10AE0000002EDDD1EB681A7859683A80200028E0DE
:10AE1000614BC018032800D979E000F0ADFD846AC9
:10AE2000789E5E4B9842B2D10B20002EC8D10123F0
:10AE30003B80EB6831001B7823706889013080B259
:10AE4000FCF7A2FF3A88031E0ED0017802328A185E
:10AE50003A80428962704289120AA2705968027867
:10AE6000E01C00F0D9FC06E004323A8031000422F4
:10AE7000601C00F039FF0020A2E70B20002E9FD1BC
:10AE8000EB6807A91E8804233B80330A3000267034
:10AE90006370FCF779FF051E28D004AB9A890E2356
:10AEA00004A95B183E49C668FCF7E2FF00280BD1F5
:10AEB0002B783C486A680599FBF798FB002803D17A
:10AEC000012304AA5B42D3813278022A06D1716839
:10AED000201D00F0A1FC3B8802333B800E2304AA16
:10AEE0009B181B88A3701B0AE370C4E704ABDE81C8
:10AEF000F4E70B20002E00D062E7E9680398FFF723
:10AF000029FF02233B802070000A6070B3E70B200A
:10AF1000002E00D054E70222EB681B883A80237091
:10AF20001B0A6370A7E7E86800F036FDC2B20300B1
:10AF30000720B24200D243E70DD00299DBB271186C
:10AF4000994202DB921BD3B20293029BE9681A007A
:10AF50003B8089195AE70023F6E70B20002E00D02A
:10AF60002EE70722EB683A801A7822705A786270CE
:10AF70005A88A2705A88120AE2701A792271DA8805
:10AF80006271DB881B0AA37175E7C04604290000C3
:10AF90000228000000D8FFFFFFD6FFFF03280000B3
:10AFA000FFFF0000F8BF0011F0B58DB06B46002028
:10AFB000089120229B5E83423DDAA64B187800F070
:10AFC0000BFE071E32D00378B02B2CD1007902384B
:10AFD00016281FD800F0B8FB17001E001E001E0028
:10AFE00031001E0096001E001D011E0052011E00B1
:10AFF00073011E00CD011E0050021E001E001E0027
:10B000008E021E00E302944B94491B8878880B80C3
:10B01000FBF72CF83800FCF7ADFF914B1B68002BB9
:10B0200001D038009847380000F08EFD8020089B42
:10B030000002434018000DB0F0BDEE220021874809
:10B0400000F052FE0BAA3B7B7989388900923A00C6
:10B050000D32FCF7B1FD0400804B1B78002C3FD172
:10B0600046E0804B788805937F4B4100CB5A0BAE6E
:10B07000073BDBB232880293002301937B4B210014
:10B0800006930093059BFFF76FFE744D002810D1C7
:10B09000069B3A8A1B889A420BD1380005991230D8
:10B0A00000F0E2FB002804D02B7862899B00EB18AB
:10B0B0005A80162306A81B18328820007989FCF7CD
:10B0C000D7FE2B7804009A00AA1851880029C3D013
:10B0D0000133DBB22B70002807D006A9C98A918002
:10B0E000634A12889A42BCD802E001214942918009
:10B0F000002B04D059497888FAF7ECFF8AE73E899B
:10B100000A2479E000253E89574B06937B88069AEE
:10B110005B009B5A033B9D4202DB002DF0D05BE0BD
:10B12000162206A812183B7B798900923A0030005B
:10B130000D32FCF741FD0590002858D04689017A70
:10B140007888FCF703FD041E44D1464B78880793AA
:10B15000069B4100C95A454B0439C9B206AAD28A96
:10B1600006930291019400930599079BFFF7FCFD5C
:10B17000041E2FD1069B39491A88931C002D26D115
:10B180004B807988384B4900CB5A5119033B8B428D
:10B1900020DD059B31485B8941190B71A91C0135E4
:10B1A000C9B2EDB2059145191B0A2B71059B2D49BA
:10B1B0000433181800F030FB2C4B059A1B88D31869
:10B1C000DDB22C4B9E4205D00136B6B29CE74988D1
:10B1D0009942D6D0002D0CD0204C2800618800F078
:10B1E0006BFC207021007888FAF784FF12E7059C39
:10B1F000F0E7002C00D183E77B78142B00D109E71E
:10B2000016493B794E800B700C717888FAF724FF51
:10B2100000E7162406ABE41821003889FCF7B4FDDA
:10B22000011E00D1B7E1788822880F4C45002C5BC5
:10B230000A4D013CE4B2029400240F4B01940095A6
:10B24000FFF792FD041E00D014E129007888FAF778
:10B2500061FFDFE6706BFF1F1C43FF1F8868FF1F45
:10B260007C68FF1F7C69FF1FB864FF1F6C6AFF1FAB
:10B270001A43FF1FFFFF00008A68FF1F162406AB5A
:10B28000E41821003889FCF77FFD011E00D182E11E
:10B2900078882288AE4C45002C5BAE4D013CE4B270
:10B2A00002947C89AC4B01940095FFF75DFD041E70
:10B2B00000D0DFE029007888FAF736FFAAE60025FB
:10B2C000A44B1D803B00F6331B78A24A7888079276
:10B2D000AB4208D99E4B12880693069943005B5AED
:10B2E000013B9A4203DB0799FAF728FF92E61624FE
:10B2F0006B00FB18059306ABE418059B2100188929
:10B30000FCF742FD011E03D1059B01241E8973E752
:10B310007888924B2288069C099343001B5B904ED1
:10B32000013BDBB20293002300960193099BFFF7D8
:10B330001BFD041E02D0059B1E895DE77B88069AD3
:10B340005B009B5A079A108832881218934202DCDD
:10B350001B1A013B33807F4C023032880999001957
:10B3600000F05AFA2388328801359B182380EDB209
:10B37000A8E70BAA3B7B7989388900923A000D3205
:10B38000FCF71AFC00250590059B002B04D10A242C
:10B39000002D00D16EE060E0059B7888197AFCF7FB
:10B3A000D5FB0100041E63D1694C6C4B7888069470
:10B3B0000993069B4400E45A694B063CE4B20BAE89
:10B3C000328807930294019100930599099BFFF736
:10B3D000CBFC041E4CD1079B5E491B881A1D002D17
:10B3E00030D14A80059B5B4C5A8963191A716B1CDA
:10B3F0009BB2E318120A1A71162306A832881B188A
:10B4000079890598FCF734FDFF21AA1C2E1D033510
:10B410000B00059092B2B6B2ADB2002803D006ABD5
:10B42000DB8AD9B21B0AA218651911712B714C4D18
:10B43000301D2A884949201800F0EEF92B88F618AB
:10B44000B5B2A1E74988914207D17A88069952009E
:10B45000525AEB18053A9A42C4DC3E4C28006188E7
:10B4600000F07AFC207021007888FAF771FED1E5AF
:10B47000002DF2D13E89BFE6162606ABF618310044
:10B480003889FCF781FC3D000400FA3500282DD0F6
:10B49000037A9B060CD400227B8939897888009234
:10B4A0003A000C32FFF7E8FB041E10D03E8915E08D
:10B4B0003088FFF741FB00281AD08368002B17D093
:10B4C0002100122278889847041EE4D0EEE72B78FA
:10B4D000002B02D17888FAF74BFE00262B78002B40
:10B4E00000D097E5002C00D194E585E60124DDE746
:10B4F0000E24DBE7162506ABED1829003889FCF78A
:10B5000043FC041E47D0037A9B0611D4154A7B885E
:10B510001188994203D01448814207D11380134BFC
:10B52000F2261D780023D9B2A94221D30924A1E72C
:10B530002888FFF701FB00282FD08368002B2CD030
:10B540002100122278889847041EDFD092E7C04677
:10B55000B864FF1F8868FF1F8A68FF1F7C69FF1F90
:10B560006C6AFF1F686BFF1FFFFF0000666BFF1F09
:10B5700031005943546801336018615A0029D2D10F
:10B580003C0008342100F22200F046F921007888BE
:10B59000FAF7F6FD3EE501246CE70E246AE71D4B41
:10B5A0001A887B889A4231D07888FAF7F3FD31E522
:10B5B000F223059851684343CD18C95A00291FD07A
:10B5C0003B7A012B0BD16C88AB887888AA1D00943C
:10B5D000FFF752FB041E02D000233B722E88F2229A
:10B5E0000021280000F080FB00232B80059B013305
:10B5F000DBB20593084B05991B78064A8B42D7D8D6
:10B6000001235B421380002CCED0F5E500263400E8
:10B610000596EFE7686BFF1F666BFF1F70B50400B0
:10B620000E001500FFF796FA031E08D131000548F9
:10B63000FFF790FA03001120002B02D01C8000209D
:10B640009D7070BDFFFF0000F8B50B4F06003B7802
:10B650000D001400FF2B0ED00A2000F0FDF9011E92
:10B6600009D0B1230380002346800371C580048183
:10B67000387800F0A9F8F8BD7144FF1FF7B50F0046
:10B6800008A90600088809A90B240988002821D1E7
:10B690000234022B1ED1557813782D021D432B0046
:10B6A0008B4301937334002B14D1FB6830001900D5
:10B6B0000093FFF74FFB019C85420BD02A0030001E
:10B6C0000099FFF7ABFF041E04D12A0030007989EE
:10B6D000FFF7BAFF2000FEBDF0B50E7885B00390ED
:10B6E0000AA805880120022E0DD14C6827786478BD
:10B6F00024023C43054FBC4205D10398DBB20196BE
:10B700000095FFF7BBFF05B0F0BDC0460229000061
:10B71000034B10B51B68002B00D09847FEE7C046CE
:10B72000746BFF1F07B501A8FFF7F2FF044A054835
:10B730000021121A00F060FAF8F79EF8FEE7C04602
:10B74000786BFF1F7444FF1F01B40248844601BC9C
:10B75000604700BF893BFF1F01B40248844601BC1B
:10B76000604700BF3555000001B40248844601BC63
:10B77000604700BF2951010001B40248844601BC62
:10B78000604700BFF30E000001B40248844601BCCC
:10B79000604700BF453BFF1F01B40248844601BC1F
:10B7A000604700BFE117000001B40248844601BCB5
:10B7B000604700BF3519FF1F01B40248844601BC31
:10B7C000604700BF8D12000001B40248844601BCEE
:10B7D000604700BF594F010001B40248844601BCD4
:10B7E000604700BF691F000001B40248844601BCE5
:10B7F000604700BFF13AFF1F01B40248844601BC14
:10B80000604700BFD91B000001B40248844601BC58
:10B81000604700BFC530FF1F01B40248844601BC29
:10B82000604700BFE94C010001B40248844601BCF6
:10B83000604700BF7918000001B40248844601BC8B
:10B84000604700BFB54C010001B40248844601BC0A
:10B85000604700BF055E000001B40248844601BC99
:10B86000604700BFA136FF1F01B40248844601BCF7
:10B87000604700BFCD4C010001B40248844601BCC2
:10B88000604700BF5147010001B40248844601BC33
:10B89000604700BF2146010001B40248844601BC54
:10B8A000604700BFC521000001B40248844601BCC6
:10B8B000604700BF2526000001B40248844601BC51
:10B8C000604700BF1D4B010001B40248844601BC23
:10B8D000604700BF056A000001B40248844601BC0D
:10B8E000604700BF9537FF1F01B40248844601BC82
:10B8F000604700BFFD19FF1F01B40248844601BC28
:10B90000604700BFEDA5000001B40248844601BCB9
:10B91000604700BFC56D010001B40248844601BC08
:10B92000604700BF8B52010001B40248844601BC4D
:10B93000604700BF5522000001B40248844601BCA4
:10B94000604700BFC51D000001B40248844601BC29
:10B95000604700BF0919FF1F01B40248844601BCBB
:10B96000604700BFADAE000001B40248844601BC90
:10B97000604700BF5D34FF1F01B40248844601BC2C
:10B98000604700BF753BFF1F01B40248844601BCFD
:10B99000604700BFAD30FF1F01B40248844601BCC0
:10B9A000604700BFDD52010001B40248844601BC7B
:10B9B000604700BFC926000001B40248844601BCAC
:10B9C000604700BFED32FF1F01B40248844601BC4E
:10B9D000604700BF4550000001B40248844601BCE6
:10B9E000604700BFD949010001B40248844601BC48
:10B9F000604700BF9536FF1F01B40248844601BC72
:10BA0000604700BFC939FF1F01B40248844601BC2A
:10BA1000604700BF1147010001B40248844601BCE1
:10BA2000604700BF753AFF1F01B40248844601BC5D
:10BA3000604700BF350E000001B40248844601BCD7
:10BA4000604700BF5139FF1F01B40248844601BC62
:10BA5000604700BFC94A010001B40248844601BCE6
:10BA6000604700BF1D4D010001B40248844601BC7F
:10BA7000604700BFED4A010001B40248844601BCA2
:10BA8000604700BF810E000001B40248844601BC3B
:10BA9000604700BF8939FF1F01B40248844601BCDA
:10BAA000604700BF5549010001B40248844601BC0B
:10BAB000604700BF1D3BFF1F01B40248844601BC24
:10BAC000604700BF350E000001B40248844601BC47
:10BAD000604700BFB352010001B40248844601BC74
:10BAE000604700BFE548000001B40248844601BC3D
:10BAF000604700BF3D18000001B40248844601BC05
:10BB0000604700BFB14E000001B40248844601BC4A
:10BB1000604700BF090E000001B40248844601BC22
:10BB2000604700BF456B010001B40248844601BC78
:10BB3000604700BF2124000001B40248844601BCD4
:10BB4000604700BF3D39FF1F01B40248844601BC75
:10BB5000604700BF434D010001B40248844601BC68
:10BB6000604700BF3D4B010001B40248844601BC60
:10BB7000604700BFCD1BFF1F01B40248844601BCD3
:10BB8000604700BF5952010001B40248844601BC1D
:10BB9000604700BFDD66010001B40248844601BC75
:10BBA000604700BF4551010001B40248844601BC12
:10BBB000604700BF4938FF1F01B40248844601BCFA
:10BBC000604700BFC9A9000001B40248844601BC17
:10BBD000604700BFC536FF1F01B40248844601BC60
:10BBE000604700BFF54E010001B40248844601BC25
:10BBF000604700BF093AFF1F01B40248844601BCF8
:10BC0000604700BFB70E000001B40248844601BC83
:10BC1000604700BFF94C010001B40248844601BCF2
:10BC2000604700BF2D33FF1F01B40248844601BCAA
:10BC3000604700BFE928000001B40248844601BC07
:10BC4000604700BF6DBC000001B40248844601BCDF
:10BC5000604700BF091B000001B40248844601BCD4
:10BC6000604700BF311B000001B40248844601BC9C
:10BC7000604700BF5D17000001B40248844601BC64
:10BC8000604700BF014C010001B40248844601BC7A
:10BC9000604700BF5125000001B40248844601BC42
:10BCA000604700BF75A9000001B40248844601BC8A
:10BCB000604700BF0124000001B40248844601BC73
:10BCC000604700BF291C000001B40248844601BC43
:10BCD000604700BF017F000001B40248844601BCF8
:10BCE000604700BF4D31FF1F01B40248844601BCCC
:10BCF000604700BF154D010001B40248844601BCF5
:10BD0000604700BF6571010001B40248844601BC70
:10BD1000604700BF9DA9000001B40248844601BCF1
:10BD2000604700BFA54F010001B40248844601BC32
:10BD3000604700BF4D1F000001B40248844601BCAB
:10BD4000604700BF0D52010001B40248844601BCA7
:10BD5000604700BF851F000001B40248844601BC53
:10BD6000604700BF090E000001B40248844601BCD0
:10BD7000604700BF156B010001B40248844601BC56
:10BD8000604700BF613BFF1F01B40248844601BC0D
:10BD9000604700BFA946010001B40248844601BCC7
:10BDA000604700BF6D2EFF1F01B40248844601BCEE
:08BDB000604700BF855201004D
:10BDB800000301020203030304030500060207004F
:10BDC800080209030A030B030C000D000E030F03FE
:10BDD8001003110313031403150216023D3C00114E
:10BDE800713C00110000000002000000FABD0011C3
:10BDF800192A0F180A000000F1590000FD2400005C
:10BE080041460100C5810011D9A100112D7600110C
:10BE1800C97F001155540011A9AF0011A15000119C
:10BE28004D3E00117D3F0011000000001616000075
:10BE38000200000044BE0011F4FFF3FFD2FC000032
:10BE4800BD40001100000000000000005475796139
:10BE58000042322E30003030314100676974687515
:10BE6800622E636F6D2F70767678005448423300E7
:10BE7800020000008CBE0011292A282A272A262A17
:10BE8800252A242A0A180000E20400007102000092
:10BE980078EC000005000000744000001027000046
:10BEA80060F000000400000006640000204E00005E
:10BEB80000000000060000005C440000102700009D
:10BEC8006CEE000007000000050000001F501D1068
:10BED800023CB40000011A0020000000A10200008A
:10BEE80030313233343536373839414243444546A8
:10BEF8000000000059580011AD5800110000000062
:10BF08000200000014BF00116F2A6E2A1A18EAD81E
:10BF1800BC80F0FC600000000000000000005F062C
:10BF28006B2F363D7D077F3F777C596E7971000016
:10BF380001A00000000000006410B71DC8206E3B7F
:10BF4800AC30D9269041DC76F4516B6B5861B24D18
:10BF58003C7105502083B8ED44930FF0E8A3D6D682
:10BF68008CB361CBB0C2649BD4D2D38678E20AA0EA
:10BF78001CF2BDBDFB349B5F8000008000100000F8
:10BF8800000000002F620011B978001153620011FF
:10BF9800C17C0011D7620011977C00114D6300111C
:10BFA8006D7C00119F630011357E0011076400113C
:10BFB800357E001139640011EF7D00114D630011C9
:10BFC800257C0011C5630011CD7D00110000000023
:10BFD80000000000AB640011CD7D00110D6500115B
:10BFE800D1780011052A042A012A002A02290328E7
:10BFF80001280028011800180000000000000000B7
:10C008000000000000000087010102010201010296
:10C0180001020303040103010101010103030201F9
:10C0280003000D000E001000110013001401070199
:10C0380008010A010B011C011D0204020502070286
:10C04800080219021A021C021D0301030203170049
:10C058000201000504000807000B0A001716001D5E
:10C068001C010201010504010E0D01111001141338
:10C07800011716011A19020201020B0A020E0D021B
:10C088001110021413021716030504030807030B03
:10C098000A030E0D0001020307090A0B0E0F101107
:10C0A80012141718191A1B1F20212200F1A80011B9
:10C0B800ADA900110000000002000000FEBF001141
:10C0C80000000000D9B600110000000002000000C6
:04C0D800FCBF001198
:020000041FFFDC
:1000000000000000B53D001100BE0011FCBD001154
:10001000A461FF1F000000000000000000000000BD
:1000200000000000000000000000000000000000D0
:1000300000000000000000000000000000000000C0
:1000400000000000000000000000000000000000B0
:1000500000000000000000000000000000000000A0
:100060000000000000000000000000000000000090
:100070000000000000000000000000000000000080
:100080000000000000000000000000000000000070
:100090000000000000000000000000000000000060
:1000A0000000000000000000000000000000000050
:1000B0000000000000000000000000000000000040
:1000C0000000000000000000000000000000000030
:1000D0000000000000000000000000000000000020
:1000E0000000000000000000000000000000000010
:1000F0000000000000000000000000000000000000
:1001000000000000000000000000000000000000EF
:1001100000000000000000000000000000000000DF
:1001200000000000000000000000000000000000CF
:1001300000000000000000000000000000000000BF
:1001400000000000000000000000000000000000AF
:10015000000000000000000000000000000000009F
:10016000000000000000000000000000000000008F
:10017000000000000000000000000000000000007F
:10018000000000000000000000000000000000006F
:100190005133FF1F9931FF1FC166010000000000AD
:1001A000000000000000000000000000000000004F
:1001B000000000000000000000000000000000003F
:1001C000000000000000000000000000000000002F
:1001D000000000000000000000000000000000001F
:1001E000000000000000000000000000000000000F
:1001F00000000000000000000000000000000000FF
:1002000000000000000000000000000000000000EE
:1002100000000000000000000000000000000000DE
:1002200000000000000000000000000000000000CE
:1002300000000000000000000000000000000000BE
:1002400000000000000000000000000000000000AE
:10025000000000000000000000000000000000009E
:10026000000000000000000000000000000000008E
:10027000000000000000000000000000000000007E
:10028000000000000000000000000000000000006E
:10029000000000000000000000000000000000005E
:1002A000000000000000000000000000000000004E
:1002B000000000000000000000000000000000003E
:1002C000000000000000000000000000000000002E
:1002D000000000000000000000000000000000001E
:1002E000000000000000000000000000000000000E
:1002F00000000000000000000000000000000000FE
:1003000000000000000000000000000000000000ED
:1003100000000000000000000000000000000000DD
:1003200000000000000000000000000000000000CD
:1003300000000000000000000000000000000000BD
:1003400000000000000000000000000000000000AD
:10035000000000000000000000000000000000009D
:10036000000000000000000000000000000000008D
:1003700025B7001100000000000000000000000090
:10038000000000000000000000000000000000006D
:10039000000000000000000000000000000000005D
:1003A0000000000000000000000000004D1BFF1FC7
:1003B000000000000000000000000000000000003D
:1003C000000000000000000000000000000000002D
:1003D000000000000000000000000000000000001D
:1003E000000000000000000000000000000000000D
:1003F00000000000000000000000000000000000FD
:08183800806FFF1F4118FF1F24
:10184000024981F3088802F0F3FB0000806FFF1F5C
:1018500070B500241E491F4A1F484C6308CA1B0567
:101860001B0DE4188242F9D11C4B80228B630021AE
:1018700009201B4B920519621A4B1B4DDA671B4B53
:10188000DA688243DA609A68194802409A60112047
:10189000296002F0B9F8112002F096F86B6C154A35
:1018A000112013406B64EE23DB006343124A1B0CD0
:1018B00013840122114B9A7201F024FC104B1B7807
:1018C000002B04D10F4B1021187802F0C9F970BD1C
:1018D000000005400806054080060540FF010000A5
:1018E00000F0004004E100E0003800403CF000401F
:1018F000FFDFFFFFFFFEFFFF7461FF1F2862FF1F76
:101900005664FF1F5462FF1F10B502F069F90728E3
:1019100004D0122808D0022808D010BD044A0420A0
:10192000136B01331363F8E70220F6E71420F4E7A2
:101930006065FF1FF8B507000C0026002500503633
:1019400030785135002804D10300287058342370B2
:10195000F8BD2978CA00481E8141A3183800A25C4E
:101960005B68C9B2FFF7D0FF00280DD12B78DA00F1
:10197000A218013350602B703378044A013B337056
:10198000136A01331362D8E70123DFE76065FF1FA5
:101990005C234343074910B5C9180B0058331B7823
:1019A000012B05D1FFF7C6FF034A936A0133936207
:1019B00010BDC0469465FF1F6065FF1F10B502F0A3
:1019C0008FF9064A0121130010CB4942D967044B15
:1019D000136002F0FDFA200010BDC04600E100E0F7
:1019E0001000100010B5040002F07AF9024B1C60E0
:1019F00002F0EEFA10BDC04600E100E010B50400B0
:101A000002F06EF94021094A200013688B431360ED
:101A100000F0F6FA01F07EFC0022054B01201A606E
:101A2000044B04321A6002F0F3F8FEE71CF00040A9
:101A3000C4F00040C0F00040431E5A425341A0226F
:101A4000F0B5D2015B421340154D164A40019B1878
:101A50002A18127E8BB00191002A1BD01A0008327E
:101A6000D46F0022E6B206AFE4B294420EDC28182E
:101A7000C369002B08D0019902AA117106AA049229
:101A800002AA167303A898470BB0F0BD1978B95491
:101A90000132EAE71A7D1A7806AB01261A70E6E7EA
:101AA0002068FF1F00400040F0B5254B04004001B6
:101AB000C25C85B0002A2BD01A18117E002927D0CD
:101AC000917E002924D01179022921D11689D78845
:101AD000D168F51BADB22A1C102D00D9102292B28C
:101AE000BE4217D11818012303710023C269C380B5
:101AF00003819A4206D06846032103730171029361
:101B000001A890470820002C00D0192001F0FAFA13
:101B100005B0F0BD013C65426C41A0256442ED0179
:101B20002C40084D1B186419074D0633013A92B238
:101B3000AA42EDD01888461C1E80085C2070F5E78C
:101B40002068FF1F00400040FFFF00000F220E4BE7
:101B500010B59868104002380A280BD802F00AF82D
:101B60000D0A0B0A0A110A0A0A0A060002210020BD
:101B7000FFF762FF10BD0121F9E70020FFF794FF96
:101B8000F8E7DB6FF6E7C046004000400F220E4B3F
:101B900010B59868104002380A280BD801F0EAFF07
:101BA0000E0A0B0A0A120A0A0A0A0600022101207A
:101BB000FFF742FF10BD01210800F9E70120FFF700
:101BC00073FFF7E7DB6FF5E70090004013B5334C88
:101BD0002378072B3DD8324B1A78324B002A39D163
:101BE0008022196852020A431A60252001F0CCFEB7
:101BF00020232D4A11680B43802113606B46042279
:101C0000C90508680733104228D080210422C9057D
:101C1000C86810422ED080212020C905CA6882439E
:101C2000CA6014221A701A78002A2FD18021C9059F
:101C3000C86820320243CA6014221A701A78002A37
:101C400028D11A4B1A7D22785A601D221A705932F7
:101C5000DA6013BD1A6816490A40C5E708680243EE
:101C60000A6014221A701A78002ACED01A78013A23
:101C7000D2B2F7E7C8680243CA6014221A70197812
:101C80004A1ED2B21A700029F9D1C4E71A78013A73
:101C9000D2B2C7E71A78013AD2B2CEE7AC43FF1FFF
:101CA0007444FF1F3CF00040A443FF1F002000408D
:101CB000FFFFFEFF564B70B51B68012B03D1554A41
:101CC000936D0133936502F09BF8534B534A1860B0
:101CD000534B544C1A600123534A1360534A136008
:101CE0002378002B06D006225149524802F028F9E9
:101CF00000232370504A514B10681B78C1B2002B4F
:101D00000ED14F4CC0B223785BB2002B4FDB23784F
:101D100024785BB264B21B0424021B191B181360E5
:101D20000B1C50294ED95023464A47491078DBB244
:101D3000FF2202284BD10868444C454D2678904339
:101D40002A78964254D9227824782E78023B5D1066
:101D5000A31B6B435201D31A10335B111843086065
:101D600002F026F9031F012B45D83A4B1B78002BB4
:101D700006D0394B1B78002B02D0002002F0A8F8C7
:101D8000A122364B92009978354B4A431B689B1829
:101D9000832292009B181B78033B012B03D8AF20B2
:101DA000400002F065F901222E4BDA8270BD2378E3
:101DB00024785BB264B2FF33FF341B0424021B1986
:101DC0000138ABE7CAB2022AAED20223ACE70868F8
:101DD000254C264D267890432A78964208D92278B9
:101DE00024782D78023B5B10641B63435201B2E7F9
:101DF0002378DBB2B2E70228D5D11D4B1B78013B1B
:101E0000022B03D91B4B1B78022BCCD16C20C8E7CB
:101E10009809FF1FFC0FFF1FAC64FF1FFF3F00006E
:101E200014100340B064FF1F0C1003400010034067
:101E3000D50BFF1F7211FF1FB40003408C09FF1F59
:101E4000680AFF1F490AFF1F94000340460AFF1F4C
:101E5000470AFF1FF908FF1F2209FF1F300DFF1F50
:101E60003409FF1FBC0BFF1F440AFF1F450AFF1F59
:101E70001C09FF1F2309FF1F10B502F069F800229B
:101E8000014B1A8010BDC046A864FF1F10B501F0B9
:101E9000C7FEA121054A89009478054A614312686A
:101EA000044B5218528C1A8010BDC046300DFF1FD3
:101EB0003409FF1FA864FF1F10B50D4B0D4A997818
:101EC000A1239B004B431268D218531DD97F0A4BA4
:101ED0001B88994209D2441C07D0C82805D0D26972
:101EE0005B1A5A43054B5343C01801F0A9FF10BDBC
:101EF000300DFF1F3409FF1FA864FF1F710200008F
:101F000070B5244D2B68002B28D001F0B9FF2B6849
:101F1000D8402B680400002B27D001F0F9FE2B6875
:101F2000D8401D4B1D4A9978A1239B004B43126852
:101F3000D118D25C91239B00002A20D0CA580132CC
:101F4000CA50174B17491B680868834214D3D23B09
:101F5000181A012A1AD0144B186070BD01F090FFB6
:101F6000124B196801F02CFFD3E701F0D1FE0F4BA3
:101F7000196801F025FFD4E70D495B18E8E7CA505E
:101F80000C4B1B68DB68E418201AE4E7F530FF30DF
:101F9000E1E7C0461C08FF1F300DFF1F3409FF1F7B
:101FA0009C09FF1FAC64FF1FA009FF1F1808FF1F3B
:101FB0002DFF3F00B464FF1F70B504000D002829F9
:101FC00016D10300A433C2881B889B1A0B4A9BB20C
:101FD00093420DD906006A3605223100653001F0C2
:101FE0008FFF002804D13100200001F0C9FE70BD30
:101FF0002900200001F04CFEF9E7C046FE7F0000FA
:10200000F8B50500012001F03BFE134CA36AA26A5B
:102010009342FBD1114E336001F0AAFE1049030038
:1020200008601048426894460F4A17680022BC4571
:1020300001D24268BA1A0D4802603268AD18A42273
:10204000E562606A520302436262094A1278002A1A
:1020500001D00F3B0B60F8BD00F00040340AFF1FB9
:10206000E408FF1F28100040180AFF1F1C0AFF1F6A
:102070001C09FF1F70B580241025E405A3682B43BD
:10208000A36001F005FFA368AB43A36070BD00002F
:10209000F7B5160080221C001023D205019191682B
:1020A00005000B43936000225A4BD7301A6001F0B1
:1020B0008FFD9D232A002F009B00EB58CA3201217F
:1020C0000092FC37002B01D00021009A386801F003
:1020D000D7FF2900009BCB311A784F4BD3351A60BC
:1020E0004B780A781B0213438A7812041A43CB7880
:1020F0001B061343494A1BBA13604B790A791B022A
:1021000013438A7912041A43CB7931001B06134317
:10211000434A1BBA13606B782A781B021343AA78D0
:1021200012041A43EB781B0613433E4A1BBA136092
:10213000019A330213433C4A13603C4B22001B1BA1
:102140009C4603293DDCB3089A0013005142B21AA1
:10215000032A46D1354AE018511A82784078120491
:1021600000020243E05C043302430A600022FF2BBA
:102170004BDDF0222E4B12011A600F222D4B1A60FC
:102180002D4A1368002BFCD00023224A27491360F4
:10219000091B321D0B191B68043A180A2370607062
:1021A000180C1B0EA070E3700434002AF2DC8022AD
:1021B00010213B68D20501333B6093688B439360E9
:1021C000F7BD6346D578981893782D061B042B43EA
:1021D000157804392B43557804322D022B430360C4
:1021E000AFE7022A0AD1114AE05C511AE21852788C
:1021F000120202430A6004339BB2B7E7012AB5D149
:102200000A4A521AE15C1160F5E7084959180A6058
:102210000433ACE7000004403C00044038000440B4
:1022200034000440300004400C000440000104402D
:10223000040004401000044014000440F7B51500E9
:1022400080221C001023D2050091916807000B43E7
:1022500093600023654AD730136001F0B9FC9D23D9
:102260003E009B00F9583B00CA363200FC3300297F
:1022700000D07FE0586801F003FF390032785C4BF2
:10228000CB311A604B780A781B0213438A78AC462C
:1022900012041A43CB78281D1B061343554A1BBA58
:1022A00013604B790A791B0213438A7912041A438B
:1022B000CB791B061343504A1BBA13604B7A0A7A38
:1022C0001B0213438A7A12041A43CB7A21001B069D
:1022D00013434A4A1BBA1360009A2B021343484A1D
:1022E00013602200474B1B1B0093009BCE785B18AA
:1022F00001938B7836061B0433430E78043833433E
:102300004E78043136023343019E33600328ECDCFF
:102310000321A808431C9B002940800003292BD1DE
:102320003849E5185E18A9786D78E35C09042D0238
:10233000294319433160030008330021FF2B2DDDB1
:10234000314B324919600F21314B19600123274964
:102350000B60304B19680029FCD006211B680B402C
:10236000042B20D080220020D20593680A318B43B1
:102370009360FEBD01217DE7022908D121495D1846
:10238000E1184978E35C090219432960D3E7012980
:10239000D3D11C495918E35C0B60CCE719481818D5
:1023A00001600433CAE7002310490B606346002B29
:1023B0000CDC3B00FC335A68102101325A60802249
:1023C000D205936801208B439360D2E7009B9B1852
:1023D0001B68190A13705170190C1B0ED37004235B
:1023E0005B4291709C440432E0E7C0460000044028
:1023F0003C000440380004403400044030000440F5
:102400000C0004400001044004000440080F0000D8
:10241000100004401400044070B5061E19D00222BA
:102420005A4B9B799343012B13D1594B1A78FF2AAE
:102430000FD15A78FF2A0CD19A78FF2A09D1DA787D
:10244000FF2A06D11A79FF2A03D15B79FF2B00D12D
:1024500099E0504B0C201A78012A08D000224E4DEA
:102460001A7029780B00093B042B01D8212070BD7C
:102470004B1F012BFAD9454CA37B042B00D982E0DA
:10248000A279032A00D97EE09A1ED2B2012A02D88C
:1024900060881F2877D9002E56D0012E73D1A088CE
:1024A0000128E3D0002907D1581E032803D801F0E2
:1024B00061FB121715122E702978481E032811D8B7
:1024C0000025364B1D602823237501F0B9FDA84275
:1024D00027D0A580CAE702212970EDE70421FBE798
:1024E0000321F9E707390129C0D82D490968C96ACC
:1024F0008906BBD52B4908780028B7D1012A01D914
:10250000002BB3D102230B708021274D2633890184
:102510002878237501F064FD80212878890101F075
:102520009FFB0123A380214B1B78002B0AD0FA22AA
:1025300080211F4B92001B8809025A431A4B1878BE
:1025400001F076FC002092E701F0CAFB2B78A68010
:10255000073B012B03D917482E7001F079FB114B73
:10256000114C1A78002A06D0802100222078890197
:102570001A7001F035FD01F02BFD80212078090251
:1025800001F02EFDDEE7122071E7C046A60BFF1F0B
:102590006B09FF1F1A09FF1F1C09FF1F4809FF1FB6
:1025A000B464FF1F2309FF1F1B09FF1F2109FF1F21
:1025B0002C09FF1F0010004010B5002901D001F0C8
:1025C000B7FB10BDF7B5604B01919978A1239B0033
:1025D0004B435E4A060014681022E418D6235B00C1
:1025E000E0583623FF33E35C00279343222B41D18D
:1025F000574B0F3A1A600760012501F011FC019B4F
:102600001880E8235B00E35C002B01D0B34258DD67
:102610000023504FFB70AD33FF33E3581A68002A94
:1026200003D09B88DB439B071DD03823FF33E35C3B
:10263000002B18D09B235B00E35C002B13D1D1331C
:10264000FF33E35CB3420EDAA4235B00E15AE018E7
:10265000090A023101F0DCFC23000122FE33013EB5
:1026600001351A87FA70E8235B00E35C002B2AD05F
:10267000A8B2FEBD03683D00002BBED081880430A7
:10268000090A023101F0C4FCD6235B00E3581F6045
:10269000B2E72300B133BA00FF339858013781887D
:1026A0000430090A023101F0B3FCE8235B00E35C6B
:1026B000BB42EEDCE822F61AED1800235200A354C8
:1026C000A6E70027F1E7200001F032FC00281FD028
:1026D000002E1DDD7319882647190193B6002000CE
:1026E00001F09EFC5A308000201840680135818836
:1026F0000430090A023101F08BFC200001F050FA8D
:10270000A3590133A351BD4202D0019B9D42E6D1A2
:10271000114BE35C002BABD095239B00E35C002BBB
:10272000A6D00E4BE15A0029A2D00D4AA35C9942D3
:1027300002D90133A3549BE700231A212000A3549C
:1027400001F056FC94E7C046300DFF1F3409FF1F0F
:1027500000140340E010FF1F5A0200007202000044
:102760005E0200000D4970B54A6E0D4CD2038B69B4
:10277000D20BA24206D80B4D0224AA4204D901F082
:102780008FFB70BD02246442E21815007E242540B0
:102790002242F4D0A3432B438B61F0E700F00040CA
:1027A0000A200000FC1C0000F8B51D4B1D4F1A78D4
:1027B000002A10D1BA7B002A02D101321A7003E03C
:1027C000032AFAD0022AF8D001F03AFC00220120B4
:1027D000154B1A70F8BD154B154D1C68154B9E789E
:1027E00001232B702878C0B200F09EFBBB7B002B2E
:1027F0000BD101F00DFBA1239B007343E41883234D
:102800009B00E41823782B70E4E7032B02D101F03E
:10281000CFF9F0E70020022BDCD101F019FCEAE748
:102820001C09FF1FA60BFF1F2309FF1F3409FF1FF1
:10283000490AFF1F300DFF1FF0B587B00EAD2F788E
:102840000FAD2D780593AC46634614000E4D0CAACF
:1028500012782E7803930D9B009201932200059B22
:10286000029701F09DFA2E70012C01D0042C08D1A2
:10287000802206498B889343054A1278D20113437C
:102880008B8007B0F0BDC0461C09FF1F6C11FF1FF5
:102890007809FF1F0B001B3B70B504003020E02BB4
:1028A0000DD81300E025493BFF3B9BB2ED00AB4246
:1028B00005D8034B200019825A8201F0B9F970BD86
:1028C0008410FF1F10B501F09BFA054B00205B68D8
:1028D000052B04D9034A5268D20200D4980810BDCF
:1028E00000100040FCE100E070B501F0F9F90D4B7B
:1028F0001B68FC33DC691D6AFFF7E4FF641984423E
:1029000004D2094B01241B68002B07D004220024A9
:10291000064B1A70064A93690133936101F058FB24
:10292000200070BDB464FF1F9809FF1F2309FF1F1B
:10293000FC0FFF1F70B50C4D2B68FC335C6A01F077
:10294000CFF9FFF7BFFF2B680025FC339B6AE31824
:10295000834204D2054B1B68AB4200D1051B01F03A
:1029600037FB280070BDC046B464FF1F9809FF1FE5
:10297000D722044B92009B5810B5002B00D09847EB
:1029800010BDC0460000FF1F10B501F0DBF8FFF7D7
:10299000EFFF2749274BCA6D274C1A4084235B0061
:1029A0001343CB65254B1B68186A01F069F9244B6A
:1029B000244A1A60244B254A1A60A022244B520054
:1029C0001A60244B187801F043FA2000224901F0E4
:1029D000A7F90023A3600233A360204B20492360A2
:1029E00003232048A36001F09BF910221E4BFF2017
:1029F0001A60802252031A60802292031A60802299
:102A000012041A6001F064FA012001F061F9FA2061
:102A1000400001F06DF9582001F02AFB134801F045
:102A2000A7FA012001F04CF9072001F019FB10BDB5
:102A300000F0004000FEFEFF14100040B464FF1FD1
:102A4000000003400180063DBC0003403408000044
:102A5000A40003404A0AFF1F71020000C3090000DE
:102A6000FFFF3F002810004000E100E0307500004B
:102A7000674E336888331B6883F3088801F0B0F928
:102A8000644A6549136800200B401360634B644A35
:102A90001B68934200D1A6E001F092FA0221614A3C
:102AA00013688B431360FFF76FFF5F4B5F4C187821
:102AB000C0B201F0FDF90023A3600233A3605C4BB8
:102AC0000120236001F0DCF80323A36001F078F813
:102AD000040001F095F9050001F072F8554B1860FB
:102AE00001F0D6FA544B1968621A531EA14200D263
:102AF00013008022D203934201D39B029B0A3268C7
:102B0000D16AC90700D471E04C491C0C09689BB21A
:102B10004C4359432402090A641803264849FC32ED
:102B200093680A6847489B1A474A076812684749EA
:102B30009B18474A9A1833409208DB190A600360D1
:102B4000042B03D9013233400A6003600E68414907
:102B5000A619300001F034F93F4F3E493B68C318D5
:102B60003B603000019301F013F93C4E30680818C7
:102B700038493060884205D9019B01333B6001F040
:102B800007F9316001F08CFA354B1B78002B0DD022
:102B900001F036F9334B621B196812188A4232D29F
:102BA0004919091B091A304801F0BAF82F4E337A37
:102BB000002B0ED001F024F9621BF168121891422B
:102BC00024D94919091B091A294801F0A9F8002339
:102BD0003372284B83F3088801F0C2F9002001F01A
:102BE000EFF901F005F801F0EBF95CE7DC01990081
:102BF0000234641A5900641A09214B438033CB40D4
:102C0000A408E41889E7FA218900CCE71A49DBE730
:102C1000B464FF1F1CF00040FFFFC1FF0C0AFF1F40
:102C2000B641210310000040490AFF1F1410004064
:102C3000C3090000100AFF1F340AFF1F380AFF1FD4
:102C4000200AFF1F280AFF1F1C0AFF1F240AFF1F5C
:102C5000C4090000710200006008FF1F2C0AFF1F5A
:102C60001C09FF1FE408FF1F00100040740BFF1F2A
:102C70003C10004000000020DC050000A022054BB5
:102C800092009B5810B5002B01D0984710BD01F061
:102C90008FF8FBE70000FF1FA122054B92009B5815
:102CA00010B5002B01D0984710BD01F081F8FBE76B
:102CB0000000FF1FA222054B92009B5810B5002B6D
:102CC00001D0984710BD01F073F8FBE70000FF1F2B
:102CD000A322054B92009B5810B5002B01D09847BA
:102CE00010BD01F065F8FBE70000FF1FA422054BB3
:102CF00092009B5810B5002B01D0984710BD01F0F1
:102D000057F8FBE70000FF1F70B501F079F84F4B53
:102D1000186001F005F90400C30702D401F020F89F
:102D200070BD00224A4B1A604A4B187801380428BB
:102D300029D800F01FFF0320181C2400200001F0F8
:102D4000E7F80128ECD0444C2378042B6ED100F036
:102D5000FFFF0028E4D001F023F9582001F088F9A2
:102D600002232370DCE7200000F09AFFE9E720004F
:102D700001F0BEF8E5E7200000F09AFFE1E720004F
:102D800000F0DEFFDDE701F013F90500012808D1AE
:102D9000324B1B78053B012B03D82000FFF76EFF59
:102DA000D1E72D4B1B78022B01D0052B20D1022D12
:102DB00028D12B4B9B7BAB431CD12000FFF76CFF32
:102DC000264B18780128BED16405BCD4244925229D
:102DD0004B7B034205D1233A13405A4253412633D9
:102DE0001A000B7D9342AED9322001F001F8AAE718
:102DF000022D07D1194B1B78052B11D12000FFF7AD
:102E000059FFDDE7012D0BD1012B03D12000FFF786
:102E10005FFF98E7062B03D12000FFF767FF92E7DB
:102E2000200000F0C5FF022D8DD1C9E7032B04D18E
:102E30000C4B987C01F014F872E7072B00D06FE779
:102E4000094B987B00F0C4FF6AE7C0469C09FF1F4E
:102E50009809FF1F9009FF1F2309FF1F1C09FF1F6F
:102E6000A60BFF1FBC0BFF1FD40BFF1FFA210A4B41
:102E70000A4A49001A640A4A5A500A4A04395A50FE
:102E8000094A08319A64094A5A50094A5C315A5031
:102E9000084ADA667047C0460000FF1F3928FF1F46
:102EA0003529FF1FE928FF1F1924FF1FA927FF1F2E
:102EB000B91EFF1F8D1EFF1FF7B50B0CFF27012248
:102EC000009300233C001E001D009446019089B22F
:102ED00062469A401000084018413618B6B2FF2FDB
:102EE00002D1012E00D19FB2009802401A41AD18C4
:102EF000ADB2FF2C02D1012D00D19CB20133102BB9
:102F0000E6D10320012E07D1012D04D1019B24011C
:102F1000E4191C700138FEBD102EFCD10238102DB2
:102F2000F9D00230F7E700008023F7B59C46264B26
:102F3000264F01932649274A274D284C284B022823
:102F40001AD1604638600868264E30408026360325
:102F50003043086001990978002909D11660224A96
:102F60002A60224A2260E02219689143A03A1BE0BD
:102F70008021C9021160F2E766463E600F68194E73
:102F80003E408027FF023E430E60019909780029E8
:102F90000DD1176001280ED1154A2A60154A22600A
:102FA000E02219689143C03A0A431A60F7BD8021B4
:102FB00089021160EEE7E0210F4A02432A600F4ABE
:102FC00022601A688A43F0E74B0AFF1FE0000340C3
:102FD000D80003409000034000000340500003402D
:102FE00040000340FFFFE3FF0280063D80450822CA
:102FF0000180063D806608220080069880550822E0
:10300000F8B51E4B80261A68002014003440324266
:1030100032D11A681A4F32431A6001223B680630D7
:1030200093433B6000F02CFE0122164D2B681E439B
:103030002E603B680A2613433B608027BF00124B7B
:103040001B683B4211D1013EF6B2FF2E09D17E2210
:103050000E4B1C682B68E40B1440934323432B60F6
:1030600005E0082000F00CFEE9E7002EEFD18022F9
:103070002B68600893432B60F8BDC046C4F0004045
:103080005CF0004018F0004068F0004060F0004044
:1030900010B500F0EDFE01215820034A00F0B0FD0C
:1030A000FFF7AEFF10BDC046600AFF1F10B57822C3
:1030B0000021034800F004FF00F0DAFD002010BDFD
:1030C000A867FF1F70B5040000F00AFE00230C2063
:1030D0000B4A010059438D18515C00290DD0A142C3
:1030E00008D1012300246B7000F08AFF00F070FF0C
:1030F000200070BD01330A2BEBD11224F6E7C04645
:10310000A867FF1F70B5040000F0EAFD0023190056
:103110001D000D4A1078002806D0A0420CD1557031
:1031200001310C320A29F5D1002B0AD100F0A0FDA3
:1031300000F04EFF002070BD5078461EB0411B18B5
:10314000EEE700F05DFFF3E7A867FF1FF7B50400A7
:103150000C20002384460E4D019267465F43E85DD4
:103160007E19A04212D000280BD10A4B9C46624621
:103170001B7808331370019B70707C557160B360CD
:10318000FEBD01330A2BE8D10320F9E70720F7E75A
:10319000A867FF1FA467FF1F8020F8B5484BC00534
:1031A0001B68C1248360474BFF251A680123134322
:1031B0004361454BA4001A68444B40211A60444BBC
:1031C0001A68444B1A60444B1A59AA431A51C52233
:1031D00092009E58AE433143802699509F583F49F4
:1031E000F6010F403E439E509E5880273602360A15
:1031F0003043985080201A5900020A4002431A5165
:1032000004341A59364E3F04324080263A431A514C
:103210001A5936061202120A32431A5108341A5940
:1032200080260A4002431A51C32292009F58B44696
:10323000AF4337439F509F58294E0F4007439F503D
:103240009F58374080263604374380269F509F582A
:1032500036063F023F0A37439F50C0221F59AF43F3
:103260003A431A511A591202120A1643C6221E5123
:1032700092009C58AC4365462C439C509C580025BA
:103280000C4020439850C72080001A58154C11401C
:10329000C02212020A431A50134B1B78DB08AB42C0
:1032A00001DC0020F8BD2378002B06D0A368002B9A
:1032B00000D0984701350C34EEE71220F2E7C04603
:1032C000A843FF1FA443FF1FB0F00040A067FF1FEB
:1032D000B4F000409C67FF1F00E100E0FF00FFFF2B
:1032E000FFFF00FFA867FF1FA467FF1F030010B5C3
:1032F0001F2809D8072200201340072404490A7810
:10330000A24313430B7010BD00230620F5E7C0460F
:10331000A467FF1F034A0449136800200B40136091
:103320007047C0461CF00040FFFFC1FF054B064937
:103330001B780A6805485B0702401B0B13430020FB
:103340000B607047A467FF1F1CF00040FFFFC1FF28
:1033500070B50C25FFF7EAFF0A4B1C780A4BE4080E
:103360006543ED18002C01D1200070BD2B78002B97
:1033700006D06B68002B00D09847013C0C3DF1E76C
:103380001220F2E7A467FF1F9C67FF1F1FB50021F3
:1033900002220B0001910091052000F051FC022354
:1033A0000B490A681A42FCD120230393039B5A1E3F
:1033B0000392002BFAD1074A1368002BFCDA0B2486
:1033C0006C442000012100F08BFD207804B010BD7A
:1033D00090C8004000C8004013B504000A4B019398
:1033E000019B002B01D1112016BDFFF7CFFF230059
:1033F0000340044205D0052000F042FC019B013B44
:10340000EDE71800F0E7C046FFFFFF0707B500F043
:1034100067FC80220821D205936A0191002B01D11B
:103420000739916202210C4A11600199481E0190EE
:103430000029FAD103311160053101910199481E2B
:1034400001900029FAD11160002B02D18022D2050F
:10345000936200F0BDFD07BD00C00040F0B52D4CEB
:1034600089B02378002B4FD1FEF7A8FA02232A4F08
:1034700003903A681A42FCD120230693069B5A1EF9
:103480000692002BFAD1254E3368002BFCDA01207E
:10349000FFF7A2FF011E02D0112009B0F0BD03000A
:1034A00003220190009005AD9F2000F0C9FB03218D
:1034B000280000F015FD02233A681A42FCD12023AF
:1034C0000793079B5A1E0792002BFAD13368002BF3
:1034D000FCDA0120FFF780FF0028DDD10398FEF71A
:1034E00081FAAA786B7811041B020B4329780B43ED
:1034F00063601300113B0A49052B07D80123934051
:10350000A3600B60012323700020C6E780231B0308
:10351000F6E7C0469043FF1F90C8004000C8004037
:103520009808FF1F1E4B30B55A6818781D4B85B0A0
:10353000D31859424B4101210093002300F0E0FBD6
:10354000194B1A4A02259A6300221A6510325A65ED
:103550008022C4219D65164B1648D202DA67890085
:103560004258154B80241A4080231B0413434350B8
:10357000642341200393E40500F006FA402000F0A4
:1035800003FA6562039D6B1E0393002DFAD103239A
:103590006362FFF73BFFA562FFF760FF05B030BD38
:1035A0009C43FF1F95FFFEF700C80040050001FF88
:1035B00004E100E000E100E0FFFF00FFF0B585B0AE
:1035C0000700FEF7FBF9022305002D4C22681A4282
:1035D000FCD120230093009B5A1E0092002BFAD1AD
:1035E000284E3368002BFCDA0120FFF7F5FE002897
:1035F00003D01124200005B0F0BD234B236002232B
:1036000022681A42FCD120230193019B5A1E019289
:10361000002BFAD13368002BFCDA0120FFF7DCFE27
:103620000028E6D1194B1F60022322681A42FCD100
:1036300020230293029B5A1E0292002BFAD1336878
:10364000002BFCDA0120FFF7C7FE0028D1D1104B78
:103650002360022322681A42FCD120230393039B98
:103660005A1E0392002BFAD13368002BFCDA01209A
:10367000FFF7B2FE041EBCD12800FEF7B3F9B9E78C
:1036800090C8004000C8004001000006A8C80040E3
:103690000180000110B50020FFF790FF10BD000071
:1036A00010B5064B18705960FFF73CFF002113203E
:1036B000034AFFF74BFD002010BDC0469C43FF1F8F
:1036C0002535FF1FF0B5040085B003920291FEF787
:1036D00075F9882263035B0B52051A438023DB05CF
:1036E0009D6A8023274F0092BA68002601901B0331
:1036F0009A420CD9F82326001B041E401C4206D017
:103700008022214B52025E6219680A431A60002D22
:103710000BD100F0E5FA02221C4B1A608023DB0576
:103720005A62013A9A6200F053FC0023039A9342D2
:1037300020D1002D0AD100F0D3FA144B03221D60D2
:103740008023DB055A629D6200F042FC8023BA6848
:103750001B039A4208D9002E06D000220A4B0C49BE
:103760005A621A680A401A600198FEF73BF9002075
:1037700005B0F0BD009A0299D2181278CA540133EC
:10378000D4E7C0469043FF1F00C8004000C000407F
:10379000FFFFFEFFF0B587B0029103920400FEF731
:1037A0000DF9019000F09CFA802302250122234E9E
:1037B000DB0535605D629A6200F00AFC204F3B68D1
:1037C0002B42FCD120230493049B5A1E0492002B0D
:1037D000FAD11C4D2B68002BFCDA0120FFF7FCFD11
:1037E000002802D0112007B0F0BD2000039A0299F2
:1037F00000F0C6FB022304003A681A42FCD12023E1
:103800000593059B5A1E0592002BFAD12B68002BBD
:10381000FCDA0120FFF7E0FD051EE3D100F060FABD
:1038200080230322DB0535605A629D6200F0D0FBE5
:103830000198FEF7D7F8E0B2D5E7C04600C00040D7
:1038400090C8004000C80040F0B5802489B0060050
:10385000FEF7B4F8E405A36A02250393029000F092
:103860003FFA0123304F3D606562A36200F0B0FB78
:103870002E4C23682B42FCD120230593059B5A1E16
:103880000592002BFAD12A4D2B68002BFCDA01207F
:10389000FFF7A2FD002803D01124200009B0F0BDDD
:1038A000244B2360022322681A42FCD12023069372
:1038B000069B5A1E0692002BFAD12B68002BFCDACD
:1038C0000120FFF789FD021EE6D11B4B03211E607C
:1038D000030001900090202000F0B2F9022322683A
:1038E0001A42FCD120230793079B5A1E0792002BF4
:1038F000FAD12B68002BFCDA0320FFF76DFD041EC4
:10390000CAD100F0EDF980230322DB053C605A6246
:103910009C6200F05DFB039B002B01D1FFF776FD5D
:103920000298FEF75FF8B8E700C0004090C800407A
:1039300000C800400100000694C8004007B500021E
:1039400001910422000A01A9FFF724FF0EBD000027
:1039500073B5050005240B4AA3005B429B18196848
:103960006B46DE1D3000FFF7A7FA022804D133783A
:103970002B55013CEFD276BD052CFCD00128FAD1A5
:103980000230F8E7140900111F2807D8012380220C
:103990008340D20591680B43936070473F2808D855
:1039A0000123802220388340D20551690B435361A3
:1039B000F3E75F28F1D80123802240388340D20505
:1039C000116A0B431362E8E71F2807D80122802100
:1039D0008240C9058B6893438B6070473F2808D8A5
:1039E0000122802120388240C9054B6993434B61F5
:1039F000F3E75F28F1D80122802140388240C905D1
:103A00000B6A93430B62E8E71F2810D8802302005B
:103A1000DB05153A1968012A06D82022914319605E
:103A200019680A431A60704701228240F6E73F286E
:103A300011D880230200DB05353AD968032A06D85D
:103A400010229143D960D9680A43DA60EBE701227A
:103A500020388240F5E75F28E5D842238022181AF3
:103A6000413B8340D205516A99435162516A0B43ED
:103A70005362D8E710B50400012813D1A0221849D9
:103A800092050B685B015B0913430B60154B164AEB
:103A900019681140154A0A431A60402219680A43FE
:103AA0001A6010BD0028FCD101000A2000F070FA55
:103AB00021000B2000F06CFAC0220A4B920019681A
:103AC0000A4340211A601A688A431A60B0220449E6
:103AD00012060B685B015B0913430B60E1E7C0460C
:103AE00014F000401CF000407F00FEFF80FD01004C
:103AF00072B6074A1368013313600422054B1A603B
:103B00000023054A13608022D2055360FEE7C046B9
:103B10007808FF1FC0F00040C4F0004005490B6862
:103B2000002B05D1044A0A6004490A60044A136064
:103B30007047C046140AFF1F841E0000380AFF1F8A
:103B4000C4F000400023034A1360034A1360034A91
:103B50001360704754F0004040F1004044F10040D1
:103B600002B4714649084900095649008E4402BC16
:103B70007047C04602B4714649084900095C4900D3
:103B80008E4402BC7047C04603B4714649084000E9
:103B90004900095A49008E4403BC704700000000E8
:103BA00001B40248844601BC604700BF5976010059
:103BB00001B40248844601BC604700BF75F80000AC
:103BC00001B40248844601BC604700BF156B010088
:103BD00001B40248844601BC604700BF894400002C
:103BE00001B40248844601BC604700BFE9270000D9
:103BF00001B40248844601BC604700BF8552010001
:103C000001B40248844601BC604700BF016701005F
:103C100001B40248844601BC604700BFA1AF000068
:103C200001B40248844601BC604700BFF9ED0000C2
:103C300001B40248844601BC604700BF116E000019
:103C400001B40248844601BC604700BF496D0100D1
:103C500001B40248844601BC604700BFC1A5000012
:103C600001B40248844601BC604700BF0D52010008
:103C700001B40248844601BC604700BFADAE0000FD
:103C800001B40248844601BC604700BF01890000BE
:103C900001B40248844601BC604700BF51B800002F
:103CA00001B40248844601BC604700BF09340100EA
:103CB00001B40248844601BC604700BFF5350100ED
:103CC00001B40248844601BC604700BFE512010010
:103CD00001B40248844601BC604700BF691101007D
:103CE00001B40248844601BC604700BF75A90000CA
:103CF00001B40248844601BC604700BF8512010040
:103D000001B40248844601BC604700BFC56D010094
:103D100001B40248844601BC604700BF6D0B01003E
:103D200001B40248844601BC604700BF2D6C01000D
:103D300001B40248844601BC604700BFE9D40000DA
:103D400001B40248844601BC604700BFF935010058
:103D500001B40248844601BC604700BF01D700009F
:103D600001B40248844601BC604700BFDD0A01007F
:103D700001B40248844601BC604700BFBD5C01003D
:103D800001B40248844601BC604700BF85C1000001
:103D900001B40248844601BC604700BF090E000020
:103DA00001B40248844601BC604700BF9D6A000020
:103DB00001B40248844601BC604700BFE917010016
:103DC00001B40248844601BC604700BF090E0000F0
:103DD00001B40248844601BC604700BFC1F700003F
:103DE00001B40248844601BC604700BFC9A9000075
:103DF00001B40248844601BC604700BF613701003E
:103E000001B40248844601BC604700BFC95C0100A0
:103E100001B40248844601BC604700BFE9F60000D7
:103E200001B40248844601BC604700BFCD0C0100CC
:103E300001B40248844601BC604700BF8B520100B8
:103E400001B40248844601BC604700BF89370100C5
:103E500001B40248844601BC604700BFEDA50000E4
:103E600001B40248844601BC604700BF4DF9000020
:103E700001B40248844601BC604700BFED68010000
:103E800001B40248844601BC604700BFE90B010051
:103E900001B40248844601BC604700BFDD3F00001A
:103EA00001B40248844601BC604700BFD1AE0000A7
:103EB00001B40248844601BC604700BF8914010078
:103EC00001B40248844601BC604700BFB70E000041
:103ED00001B40248844601BC604700BFED6B01009D
:103EE00001B40248844601BC604700BF3D71010037
:103EF00001B40248844601BC604700BF053401009C
:103F000001B40248844601BC604700BFCD4C0100AB
:103F100001B40248844601BC604700BF013401007F
:103F200001B40248844601BC604700BFBD0B0100DC
:103F300001B40248844601BC604700BF71B0000074
:103F400001B40248844601BC604700BFE94C01004F
:103F500001B40248844601BC604700BF8D82000066
:103F600001B40248844601BC604700BF7997000055
:103F700001B40248844601BC604700BF8D110100B6
:103F800001B40248844601BC604700BF957301003C
:103F900001B40248844601BC604700BFA9A30011D8
:103FA00001B40248844601BC604700BF6DF60000C2
:103FB00001B40248844601BC604700BFDD0C01002B
:103FC00001B40248844601BC604700BF016C010097
:103FD00001B40248844601BC604700BF9DA90000AF
:103FE00001B40248844601BC604700BFB3520100DF
:103FF00001B40248844601BC604700BF53B90000C9
:1040000001B40248844601BC604700BF21A90000FA
:1040100001B40248844601BC604700BFC1150100DD
:1040200001B40248844601BC604700BFD9B000001B
:1040300001B40248844601BC604700BF2DB700119F
:1040400001B40248844601BC604700BFA9D8000003
:1040500001B40248844601BC604700BF19FA000061
:1040600001B40248844601BC604700BFF90D01005D
:1040700001B40248844601BC604700BF79120100C8
:1040800001B40248844601BC604700BF21440000DF
:1040900001B40248844601BC604700BFC16601000C
:1040A00001B40248844601BC604700BFD54401000A
:1040B00002000000FABF001101000000F0BD001175
:1040C00002000000F6BF001101000000F040FF1FD9
:1040D00002000000F8BD0011010000002462FF1F73
:1040E00002000000F4BF0011030000009861FF1FF0
:1040F0001200000002000000FABF001101000000E1
:1041000038BE001102000000F6BF001101000000DF
:1041100035BE00110200000042BE00110300000085
:10412000D361FF1F02000000F4BF00110300000074
:10413000E861FF1F02000000F6BF0011010000004F
:1041400034BE00110200000040BE00110300000058
:10415000A961FF1F02000000F4BF0011030000006E
:10416000CA61FF1F02000000FABF00110100000039
:1041700078BE001102000000F6BF0011010000002F
:104180003942FF1F020000008ABE0011010000003A
:1041900073BE001102000000F6BF00110100000014
:1041A0003842FF1F0200000088BE0011010000001D
:1041B000F061FF1F02000000F6BF001101000000C7
:1041C0003742FF1F0200000086BE00110100000000
:1041D00063BE001102000000F6BF001101000000E4
:1041E0003642FF1F0200000084BE001101000000E3
:1041F0005EBE001102000000F6BF001101000000C9
:104200003542FF1F0200000082BE001101000000C5
:1042100059BE001102000000F6BF001101000000AD
:104220003442FF1F0200000080BE001101000000A8
:1042300054BE00110202020202020000000000004F
:104240000D0C0000D94C00119F4C0011E8BE00116C
:1042500090011D0018001800FFFF0701020304056C
:10426000060201060000000000000000000000003F
:10427000000000000000000000000000000000003E
:104280000300000002000000FABF0011010000005E
:1042900008BF001102000000F6BF0011010000007D
:1042A000F442FF1F0200000012BF001101000000D5
:1042B0001E62FF1F02000000F4BF00110300000097
:1042C0008864FF1F02000000F6BF0011010000001B
:1042D000F442FF1F0200000010BF001101000000A7
:1042E0002062FF1F02000000F4BF00110300000065
:1042F0008064FF1F120000000058004015160000E7
:104300000001000000000111FFFF00005048593675
:1043100000000000000000000B000500F00000009D
:10432000B4000028002800283075A000A000A000DC
:10433000A00000080008E001F000100010001000CC
:10434000100010001000500050005000100010002D
:10435000D0070000000000000F00010005003075CC
:1043600007001000010081FF00000000FF000000B6
:10437000917500119973001129710011FFFF01005F
:10438000FF000000AD9F0011299D0011419C00110C
:104390000000000000000000000008000400000011
:1043A0003B0001085902E00188212800FF000000BD
:1043B00002000000FABF001101000000C0C000119F
:1043C00002000000F6BF0011010000002D44FF1F95
:1043D00002000000F2BF0011010000006068FF1F32
:1043E00002000000F6BF0011010000002C44FF1F76
:1043F00002000000F0BF0011010000002A44FF1F6E
:1044000002000000F6BF0011010000002844FF1F59
:1044100002000000EEBF0011010000002044FF1F59
:10442000180018001D0090010200000302020000A5
:1044300002000000FABF001101000000D4C000110A
:1044400002000000F6BF0011010000007044FF1FD1
:1044500002000000ECBF001100000000000000009E
:1044600002000000F4BF0011030000008068FF1F7D
:0244700020FF2B
:040000051FFF184180
:00000001FF
